:10000000F01F0010A56B0000A36B0000A36B0000A5
:10001000A36B0000A36B0000A36B000000000000B6
:10002000000000000000000000000000A36B0000C2
:10003000A36B000000000000A36B00005D33000014
:100040005D3100005D3100005D3100005D31000078
:100050005D3100005D3100005D3100005D31000068
:100060005D3100005D3100005D3100005D31000058
:100070005D310000A16B0000A16B0000C100000019
:10008000F933000011340000113600002936000059
:10009000A16B000071370000A16B0000A16B000094
:1000A000A16B0000A16B0000A16B0000A16B000020
:1000B000A16B0000A16B0000A16B0000A16B000010
:1000C000594A10B5136801331360584B584A1B68DE
:1000D000DBB2302B00D176E018D8182B5AD005D8D7
:1000E000082B37D0102B46D0082351E0202B00D10D
:1000F0007AE0282BF8D14F4B4F491868096888429D
:1001000052D21968481C18604C4B48E0482B00D16B
:100110006AE00AD8382B60D0402BE5D1484B1968EB
:10012000042301295DD11360DEE7502B66D0582BE4
:10013000DAD14448444B1B680168DBB24C1C0460B4
:10014000424843540221424BFF3119608023F13968
:10015000DB0530E00021374B19601968481C186036
:10016000364B5B5C3849DBB20B60282313600122FD
:10017000374B1A6010BD0021324B19602D490B68B6
:10018000581C08602D49CB5C2F49DBB20B6028233B
:100190001360EFE727490B68581C086027495B5C30
:1001A0002949DBB20B609FE7254B19688023DB05EB
:1001B000002902D02021196096E702202449FF304F
:1001C00008601021F7E780231021DB051960082360
:1001D000136081221E4B5200CBE782211C4B490049
:1001E000E9E78021C905DDE780231021DB051960DF
:1001F000082313600422164BFF32BAE71149124B51
:100200001B680868DBB2441C0C60104C23540C4B78
:100210001B680868013B0421834202D98023DB0567
:10022000C9E7116060E7C0460806001004000040FE
:100230001800004004060010FC050010D405001052
:10024000E80500100006001008000040EC05001052
:10025000E405001002231B4A70B511681A4D0B43C8
:1002600013602023194A040011680B431360184BD4
:100270001A682A401A600122186810431860154B4A
:1002800019682940196019680A431A606C22124BD8
:1002900012491A60124B186806F056FD114B18608F
:1002A000114B1860022C02D1A022104B1A60802240
:1002B0000F4B12021A6080234022DB0501201A60D6
:1002C00070BDC04604800440F8FCFFFF80800440FD
:1002D000304004403440044018000040400D03000A
:1002E0009804001014000040100000400C00004072
:1002F00000E100E00000000000000000FFFFFFFF41
:10030000202303490A681A42FCD0024B1860704748
:10031000148000400080004070B504000D002900EA
:10032000200003F017F8024B1B68002BF7D170BDBB
:10033000B405001010B503F03FF810BD10B5002053
:1003400002F02CF801F0F8FF10BD00007FB50500A9
:1003500000200C0002F0C8F9002801D003F0F4FDE1
:10036000002323602B60174B1E78002E28D121001C
:10037000280002F0E7F9300002F0B6F9002807D0B3
:1003800003F0E2FD2660210028002E6002F0DAF979
:100390000D4B1B78002B13D00C4B2A6818680C49A6
:1003A000824203D120680D68A84209D01A602368F0
:1003B00001A80B60074903F00BFC01A803F0BEFC89
:1003C0007FBDC04664020010740200105C02001081
:1003D000600200101C72000070B504000D00FFF7F1
:1003E000B5FF094A1368002B09D0013B1360032BAA
:1003F00006DD064B1B682360054B1B682B6070BD38
:1004000000232B602360FAE77002001068020010DE
:100410006C0200100023034A1360034A1360034A6E
:10042000136070476C020010700200106802001028
:10043000002310B50B60036002F084F910BD0000CA
:1004400010B5012403F046FD0C4B0020196803F0A1
:1004500055F9002003F042F9002003F01FF9084B82
:1004600020001C60074B196889B203F00DF82000CA
:1004700002F0FAFF200002F0D7FF10BDA004001028
:10048000D00500109C04001037B50C240321012076
:1004900002F060FF684601A9FFF79EFF009D002D56
:1004A00002D1013C002CF1D1FFF7CAFF002005F07A
:1004B00021FC28003EBD10B5002003F0FFF801200C
:1004C00002F0C2FF03F00CFD10BD000070B50D007E
:1004D0000400FFF7B5FFF8230121064ADB00D150E5
:1004E0002000290005F00EF9FFF7E5FF04F0FCFFFE
:1004F00070BDC046B806001070B504000D00FFF7CF
:100500009FFF0822074B29001C60074B20001D603D
:10051000064B1A6005F0F6F8FFF77CFFFFF7CBFFFC
:1005200070BDC046680200106C020010700200101E
:1005300010B50400FFF784FF200005F0B1F80400B7
:10054000FFF7B9FF200010BD10B50020FFF7F0FF46
:1005500010BD37B504000025FFF7F6FFA54203DB09
:10056000FFF7F2FF00983EBD0321062002F0F2FEE5
:10057000684601A9FFF730FF009B002BF0D1013541
:10058000ECE7000010B502000249034803F015FB38
:1005900010BDC0462A7200002F720000F0B5354B26
:1005A00085B01B6800900193002805D0019B002BAB
:1005B00002D0002002F000FB01F089FE002001F0D3
:1005C000EDFE01F0B9FE2C4C032223680221013319
:1005D00023602A482A4B01F0E5FF2368FA26013BF5
:1005E000236001F0E1FEFFF7AFFF2648FFF7CAFFE7
:1005F00096230024244D9B002B60B60003F08EF957
:10060000002807D002F06CFC00242B680134A342C0
:10061000F4DC1AE0009B002B27D01C4F3100386817
:1006200006F092FB6423584302F0AEFE02F01AFD7E
:100630003100386806F088FB02F0A6FE03A902A884
:10064000FFF7CAFE029B002BDFD0009B002B05D0DA
:10065000019B002B02D0012002F0AEFAFFF774FFDD
:100660000B4803F0AAFA05B0F0BD0A2002F0A4FE80
:10067000E4E7C046200000101800001037720000A8
:10068000EC8A00004672000030020010980400104E
:100690004C7200001A4B73B504001A49186806F032
:1006A00053FB194B194A1A490090200003F090FAA5
:1006B00002F02EF9002812D002F048F9FA21890040
:1006C000060006F041FB0500200003F0E5FA114B9F
:1006D0002A006B4310499B19201803F079FA200077
:1006E00003F0DAFA0D4B0E4A1B682018002B02D0DB
:1006F0000C4A00DB0C4A0D4903F06AFA73BDC04690
:100700009804001040420F005D7200002A72000041
:100710006172000018FCFFFF6E720000940400106C
:10072000577200005A720000878B00007972000037
:1007300070B50D0006001400002001F02FFE01F03E
:10074000FBFD310028000022054B01F02BFF0922A0
:100750000121044B200001F025FF01F025FE70BDB2
:10076000EC8A0000D48A000007B5144A144901201D
:10077000FFF7DEFF642002F01FFE72B60021114B6E
:10078000114A196001231360116013601168194246
:10079000FCD00E4A6846136080230D4A5B02116844
:1007A0000B43136080230B4A11680B4313603923FA
:1007B00001A90093084B984707BDC046817200000D
:1007C000907200007080044074800440788004407F
:1007D0008080044038820440F11FFF1F00B5084BA1
:1007E000084A89B01B7868461278074903F0F0F987
:1007F00069460120054AFFF79BFF09B000BDC046CE
:100800001500001087040010A3720000B1720000F0
:10081000F0B52C4C2C4D237885B001932F78002611
:10082000FFF7DCFFFFF790FE02A803A9FFF7D4FD56
:100830000298002815D0C0B201F0D2FE492805D890
:100840003F281ED830282CD0392835D001F060FD43
:10085000FFF7C4FF029E002E03D0C82002F0ACFDBB
:100860000026032104200136FFF756FD1E2EDBD1A2
:10087000019B2F70237001F04BFDFFF765FE05B063
:10088000F0BD40380928E1D806F0ACF905F2E0E007
:10089000E0E0F7E0E0102B783E2BD7D801332B7047
:1008A000D4E72B78002BD1D0013BF8E72378062B37
:1008B000CCD801332370C9E72378002BC6D0013B85
:1008C000F8E7C046150000108704001010B590B07E
:1008D0006846FFF7DFFE002001F060FD01F02CFD0F
:1008E0000122084C11002300684601F05BFE230042
:1008F00009220121044801F055FE01F055FD10B018
:1009000010BDC046D48A0000C572000000B52B227D
:100910008DB0002800D1023268460D4903F058F925
:1009200004A803F0A1FB6946012004AAFFF700FF19
:1009300003200021FFF7F0FC0220FFF7F9FD00285B
:10094000EED000210A20FFF7E7FC0DB000BDC04645
:10095000DF720000F8B5040016000D00002703F058
:1009600083FB2100E7741431681C03F09DF9380003
:1009700001F014FD01F0E0FC3A00042120000A4BD4
:1009800001F010FE094C092223000421280001F087
:1009900009FEBE4205D0230009227821044801F057
:1009A00001FE01F001FDF8BDEC8A0000D48A0000D0
:1009B0003175000030B58DB0134902A803F074F909
:1009C0002E24002202A904A8FFF7C4FF0025FFF788
:1009D000BBFDFF34002202A904A8FFF7BBFF0321DF
:1009E000002002F0B7FC684601A901950095FFF7C9
:1009F000F3FC009B002B02D1013C002CEAD1FFF755
:100A0000A3FD0DB030BDC04699AC0000F0B5002488
:100A100091B020009626039401F0C0FCFFF794FDEE
:100A20000223270000940193760001F085FC009BCF
:100A3000002B00D0ABE008AD280003F015FB009BB5
:100A4000EB742B746B73AB72EB712B71002C01D1B7
:100A5000012F05D10022042128008F4B01F0A2FDB7
:100A60008D4D00222B001E218C4801F09BFD012C96
:100A700001D1012F07D11D202B0002AD002225211D
:100A8000401901F08FFD844D00222B003321834853
:100A900001F088FD022C6FD1012F6DD0232002AD13
:100AA00000224D217C4B401901F07CFD7A4D002243
:100AB0002B0059217A4801F075FD042C01D1012F3A
:100AC00007D126202B0002AD00225F21401901F042
:100AD00069FD714D00222B006C21714801F062FD0F
:100AE000052C01D1012F07D129202B0002AD0022B6
:100AF0007221401901F056FD09220421694B0DA80D
:100B000001F050FD01F050FC039B002B07D0143B7B
:100B1000012B41D8052C3FD0962002F04DFC03213B
:100B20000800FFF7F9FB002001F0DEFD00230500BF
:100B300004A903A804930393FFF74EFC039B002B27
:100B400000D199E006AE05AD3100280007AA03F0F8
:100B5000BFFA0090002828D1280003F09FFB07006F
:100B600003981238052800D97EE006F045F8217D6B
:100B700056237D181E0058E72B0000223A210AA8B0
:100B800001F010FD032C89D1012F8FD186E70022BF
:100B90000421414B4448B3E7FFF7D6FCBFE7601C94
:100BA000062106F0B7F900270C009626760067E0CC
:100BB000601DF5E7601E042804D806F01DF80D142A
:100BC0001D2647002B88013300242B80280003F0CA
:100BD00065FB0523070016E00C21A87806F0B0F8A5
:100BE0000131A970F2E701372900380003F088FBD2
:100BF0000523022401932BE030780130182106F000
:100C000089F904233170019322E0707801303C218E
:100C100006F080F903237170F5E7601E042804D8FC
:100C200005F0EAFF060C0E1114002B88013BCBE700
:100C3000A8780C210A3006F06DF9D1E7013FD3E71F
:100C400030781730DAE770783B30E0E70023B37094
:100C50000721380006F05EF90A000791052C05D13E
:100C60003100280003F08CFA01279EE731002800AC
:100C7000019B03F045FAF7E7002D01D101235F4006
:100C8000039B842B05D0182B03D0731E002E00D09D
:100C900070E711B0F0BDC046EC8A0000E8720000B9
:100CA00038730000D48A0000EA720000114B10B5BE
:100CB0009A6D032A1AD11C00BB3460782278A1787F
:100CC000000210430904E27808430B49120602436C
:100CD0008A420BD1BA3318780F23034000090F2B37
:100CE00003D00F2800D00A33180010BD0120404265
:100CF000FBE7C046B8060010AFACEAFF0F210C4B73
:100D00000C4A985C0C4A9A5C0A40013AD2B200281C
:100D100008D0062A09D8083941435B189B189C3330
:100D20001878704701204042FBE70220FBE7C046ED
:100D3000B80600109507000096070000030003485E
:100D4000062B02D8024A9B0098587047878B0000F8
:100D5000F47500000300501E70B50D001D4C0328F3
:100D600003D805F049FF0B18222C18000E221A494F
:100D7000CD3402F038FF23782B7070BD18000021AD
:100D800003F096FB2300CF331B78CE341B0122786F
:100D900012091343F0E71800012103F089FB230037
:100DA000D0331B78CF341B01F1E71800022103F088
:100DB0007FFB2300D1331B78D0341B01E7E71800F9
:100DC000032103F075FB2300D2331B78D1341B01C0
:100DD000DDE7C046B8060010F0060010CB10C05C7E
:100DE000072319400841063B1840704710B5010021
:100DF0000148FFF7F3FF10BD69770000831F10B5AE
:100E00000020032B02D80248FFF7E8FF10BDC046C0
:100E100069770000002370B504000D001600037010
:100E2000292912D8094B8A00D15802F03DFF0C2D18
:100E300005D1200002F030FF201805F043FE002EFF
:100E400003D02000024906F0C3F970BD907700007E
:100E5000F872000010B50022FFF7DCFF10BD70B57E
:100E60000025040008001100AA420EDB28225A4384
:100E700052185200115F4B1C07D0A94207DA022317
:100E80005B42591AFFF7E6FF0125280070BD05F007
:100E90007DFEF9E7F8B505000E00171E0BD105F031
:100EA00087FD041E1BD131001148FFF797FF002872
:100EB00015D02000F8BD012A11D105F079FD041EDE
:100EC0000DD13000FFF792FF002808D02800220043
:100ED0000621FFF79FFF280002F0DEFE2D183B00E1
:100EE000320029000348FFF7BAFF0400E1E7C046DB
:100EF0006E770000107600001FB50D4B1B78002B9D
:100F00000AD1FFF7FBFE0100431C05DB431C05D1A2
:100F10000848023105F090FB05B000BD684605F0B9
:100F200035FE6B461B78002BF6D001216846F1E7B1
:100F300058020010FA72000010B504F0F1FE00280B
:100F40000BD0002001F02AFA01F0F6F9FFF7D4FFE8
:100F500001F012FA012001F021FA10BD70B52D4BFD
:100F600086B01B78002B05D105F046FD002803D084
:100F7000FFF7C2FF06B070BDFFF798FE041E08DB46
:100F800005F056FB2000FFF7D9FE022105F054FBC7
:100F9000F0E76B460122D91D02A8FFF7DBFE05F042
:100FA00039FDC5B205F058FD1B4EC4B20E2231000A
:100FB00002A806F0E9F8002813D1184B1A78184B4C
:100FC0005B6D9A420DD1174B1B78AB4209D1164B82
:100FD0001A786B46DB799A4203D1144B1B78A342F3
:100FE00014D00E2202A9300002F0FDFD0C4B02A825
:100FF0005A6D0A4B1A700B4B0D4A1D706B46D9790E
:10100000094B1970094B1C7005F076FC084805F077
:101010002FFBAFE7580200104602001054020010E8
:10102000B8060010550200105602001057020010BA
:101030003402001010B504F073FE00280BD000201D
:1010400001F0ACF901F078F9FFF788FF01F094F9AD
:10105000012001F0A3F910BD10B5FFF7EBFF10BDA3
:101060001121044ADC3213788B43034909780B437E
:1010700013707047B806001045020010024B187834
:10108000C006C00F7047C0464502001070B504008E
:101090000D0000200C2C09D8FFF7F0FF002806D027
:1010A00029002000FFF7AAFE431E984170BD0B4B9C
:1010B0000B4A1B5D29009B009858FFF78FFE012308
:1010C000002808D1074A12781A42EFD1252DEDD118
:1010D000054B185DEAE71800E8E7C0468077000096
:1010E000000000104502001073770000F7B50E00F5
:1010F0000500140005F0C6FC0700010000222800CE
:10110000FFF788FE31003800FFF7C0FF0190002C88
:1011100006D131003800FFF771FE431E9841C4B27A
:10112000019B002B10D00122164B28001B78134086
:10113000013B1C4002F0B0FD220031002818FFF7EF
:10114000A9FE04002000FEBD0F49280006F040F86B
:10115000280002F0A1FD220031002818FFF79AFEB6
:10116000041EEFD131000948FFF738FE041EE9D014
:10117000280002F091FD32002918019B0448FFF776
:101180006EFEDFE745020010037300006477000085
:101190000077000010B5FFF771FF0122011E074C18
:1011A00005D0074B53331A700023237010BD2378EA
:1011B0001342F9D07820FFF789F9F5E745020010CE
:1011C000B8060010F0B5050087B0002901D0012451
:1011D00012E005F017FC041EF9D1344E3278382D98
:1011E0000DD110231A4053425A4112013270FFF7B9
:1011F00037FF01222E4B1A70200007B0F0BD0127E7
:10120000782D07D13B0093433370FFF729FF284B1C
:101210001F70F1E73A4053000193FFF72FFF0028BA
:1012200000D00197280005F0CFFB070005F0C0FBB8
:101230006B4639001A79002812D002A8FFF756FF32
:101240000028C4D005F0D8FB00280DD0FFF7A2FF7E
:101250000122174B002128001A70FFF737F9CBE75E
:1012600002A8FFF717FEEBE70620FFF761F9002859
:1012700004D102A805F002FB01F096F82A20FFF73E
:1012800057F9041E07D0FFF785FF00212800FFF75C
:1012900033F90024B0E7074805F0F0FA01F084F8CC
:1012A0003470FFF7DDFEFFF74FF9A5E745020010A8
:1012B000640200100573000010B5002802D1FFF78A
:1012C00053FA10BD002001F069F801F035F8012251
:1012D0000A4C012123005242094801F063F923001E
:1012E00007220121074801F05DF901F05DF878203F
:1012F000FFF72FF98428E4D1E1E7C046DC8A00003B
:101300000A7300001C73000070B504000D0000F0AB
:10131000DEFF262C13DC0020102C27DD20001138E6
:10132000152814D805F068FC1D132D6D373F4E139A
:101330003113131313131313264213131345442CA1
:1013400054D006DC372C58D00120382C56D0002041
:101350000CE0452CFBD1E120000102F02BFF012025
:1013600048E02A4B1B68002B01D1012070BDFFF71C
:1013700021FBFAE7254B1B68002BF6D0FFF746FB55
:10138000F3E70120FFF70AF9EFE70120204B1B6884
:10139000C01A01F011FC0120FFF798FAFFF7D4F80A
:1013A000FFF772F8E1E7FFF733FADEE704F0A8FC95
:1013B000DBE70022174B1A70174B05321A7000F04A
:1013C000A7FFD2E704F0ACFC144B002806D0196844
:1013D0000322022900DD00221A60C6E71A68511CA8
:1013E000062A01D01960C0E71860BEE70C4802F079
:1013F000E1FE0020FFF78AFAB7E7002004F08AFC3C
:10140000B3E72800FFF758FFAFE7C0469404001089
:10141000200000108704001015000010A800001024
:10142000F0F1FFFFF8B5012706000C00002000F0E6
:10143000B5FF00F081FF0B4D7F422B003A000121E8
:10144000094801F0AFF82B003A0030002A2101F0E2
:10145000A9F82B0007220121200001F0A3F800F0D9
:10146000A3FFF8BDDC8A000033730000030010B551
:1014700003480449002B00D09968FFF7D3FF10BD43
:10148000878B00003A730000F0B5002787B000F0AA
:101490001EFF2A4D2A492800FFF7C4FF3C00FFF732
:1014A00053F80C260321062001F054FF684601A9D9
:1014B000FEF792FF0098002804D10137772FF1DD65
:1014C00007B0F0BDC0B201F08BF80200462808D08A
:1014D000002C0AD00023E356834206D10020205678
:1014E000EEE7002CFAD10027DCE7352A01D0412AAB
:1014F00021D114481449FFF795FFFFF725F8002084
:10150000DEE7934206D124182000FFF7AFFFFFF774
:101510001BF8E8E70131300048432356002BF0DC8C
:10152000F1D00A4902A802F053FB28000849FFF74E
:1015300079FF0024EBE70021064CECE7878B0000E5
:101540003A73000059730000467300005B7300009B
:101550006273000038780000F0B51D00070013002A
:101560000400160085B015372B4305D11B4902F046
:101570009BFB012005B0F0BD002343752000163011
:10158000C31B174A019330000023290005F0E0FC3B
:1015900000230290039130002900114A05F0D8FC85
:1015A0001300002D02D10F4A964208D9073F0722A7
:1015B0003021380002F0D5F9029E039DDEE72A00B3
:1015C0002021200002F0CDF905003900019A2018F1
:1015D00002F04CFB019B681EC018CBE7747500003D
:1015E000809698007F969800F7B51D00089B140020
:1015F00006005A1E0120002105F09EFC0B0002008F
:1016000019002300100013402A000A4013431BD086
:101610002D23337001225242D317801859410122E1
:101620000023001849418018594100900191009F02
:10163000013667403800099C019F6F40E51739006B
:10164000A41A9D4124184D412B0030002200FFF7C1
:1016500083FFFEBDF7B5009203220193099B00268C
:101660000333DC171440E418A41005192F00013FC0
:10167000A64202DB00202870FEBDB200009801994E
:1016800005F04EFC0F231840024B01361B5C3B70EB
:10169000EDE7C0466D730000F7B50193099B0400A8
:1016A0000321981C009205F04FFB24180500270029
:1016B0000026013FAE4202DB00202070FEBD032267
:1016C00000987243019905F02BFC07231840303035
:1016D00038700136EDE7F0B5069D0400142D03DDEA
:1016E0009F2114250170013400206E1EA619854229
:1016F00002DC00206055F0BD01218140CF171F4062
:10170000114039434F1EB94147423031F155013044
:10171000EDE703001A000800002130B50D321578FE
:10172000040F09010001214328431400013AA34298
:10173000F5D130BD022210B53C21024B524200F0DF
:1017400031FF10BDD48A000070B5C5B2CCB22800FC
:101750002100013400F090FE2800E1B200F08CFE80
:1017600070BD0000F0B587B00591039002F094FAC7
:101770000625431E4543070005991800049305F00C
:10178000E3FA0023013D400040190193842802DD63
:101790002800013301934B240025241AE3432E0033
:1017A000DB171C40BD4201DB07B0F0BD039B0722E5
:1017B000585D2100144B00F09DFEA31D0293039B76
:1017C0005B5D303B162B01D9002E12D0049B012605
:1017D000AB420EDD781E0599401B05F09BFB0029EE
:1017E00007D1019B002B07D0601D0631FFF7ACFF2E
:1017F000019E029C0135D5E70E2102980834FFF7BF
:10180000A3FF0294F5E7C046DC8A0000F0B5002093
:1018100093B000F0C3FD00F08FFD05F0FBF80F243E
:10182000039005F0FFF802ABE418002221000290BB
:1018300006A8FFF78FFA217806A8FFF76AFF0C00C9
:10184000050005F0F7F80600032005F00DF96B46DA
:10185000C7B2187B08282ED805F0CEF9052D392DF2
:10186000442D2D2D11002548FFF764FF2A00230089
:10187000019600970AA8FFF7EDFE04210CE020482E
:10188000FFF758FF6B461B7A002B16D12A00230066
:101890000AA8FFF761FE03210AA8FFF763FF00F023
:1018A00016FD00F069FD012000F078FD012004F034
:1018B00021FA00F079FD13B0F0BD6B46187A2A00CA
:1018C0000190230000960AA8FFF78EFEE3E70D487B
:1018D000FFF730FF2A002300019600970AA8FFF7C0
:1018E000DBFECAE70848FFF725FF2A002300019620
:1018F00000970AA8FFF7EFFEBFE7C0467E7300001F
:10190000877300009073000099730000F0B58DB0EC
:1019100002F040FB012004F0FDF9F8270021182017
:10192000FEF7D4FD0024814EFF00FEF7C4FD002326
:101930007F4DEB51200002F04FFB002C61D00121C4
:10194000002001F007FD200002F040FB03A9030086
:10195000019002A8002B57D0FEF76AFD01230193E6
:10196000002C13D002F037FB029B182B02D0019BF6
:10197000002BDAD000206F4B187000F00FFD00F044
:1019800029FD6D48FEF7FEFD0123EB6602F06CFABF
:10199000029E182E0DD1002C6FD0039BD8B200F000
:1019A0001FFE0121FFF7B0FCE851002801D0002301
:1019B000039303990298FFF705FC002807D0FFF76F
:1019C000E9FBFEF73DFD0399029803F09BFE002220
:1019D0005A4B1A70EB59934201D0FEF7B5FD94357E
:1019E0002B685C425C41002B65D100F059FC544BE4
:1019F0001A78002A03D000221A70FEF7A5FD4B4E7C
:101A000093E7032106209CE7FEF712FD029B002BC3
:101A1000A6D1002C8ED14B4B1B68002B8AD12B00FA
:101A200098331B68002B1CD1474B0024F61881D536
:101A3000464B1B78002B0BD0454802F07FF9642001
:101A400001F0BAFC434802F079F9642001F0B4FCDB
:101A500000F026FC2B00002294330224334E1A603F
:101A600068E73D4A13681133136003F0F5FD029BEC
:101A700001330293102BF8DDD6E7FFF7FFFA0028B9
:101A800097D02C4B300021001C70FEF71FFDFFF794
:101A9000FBFC0394061E8CD02100FFF735FC0028C8
:101AA00087D1F0B200F0B8FD0390482E81D001221A
:101AB0002A4B1A707DE700F05FFF002000F06EFCFB
:101AC000002500F039FC04F09DFFA84204D104F089
:101AD0006FFF431E9841050001263000684004F066
:101AE00067FD04F01DF9002806D0FFF737FA00F073
:101AF00043FC300000F052FC002D0DD004F0C2FF7A
:101B000004AD010001222800FFF784F92B78002B97
:101B100002D0280004F0BDFE04F074FF002801D1BB
:101B200004F0F0FC00F040FC61E7C04620BF02007A
:101B3000B806001045020010B673000058020010ED
:101B400064020010B40500100CFEFFFF74020010C8
:101B5000A2730000AC73000014060010D40E001035
:101B600073B54A4C4A4B22684A4D9A4202D12560CD
:101B700001F0C2F82368AB4201D10023236007269D
:101B800002F0CCF800F070FD0021434801F038FA73
:101B900001250021414801F033FA00F045FE00F034
:101BA000E9FF00223E4C100023680B21B343236061
:101BB00023682B43236001F0B5F92000394C102134
:101BC00001F01EFA23680022B34323602368280033
:101BD0002360042101F0A6F90021200001F010FA91
:101BE00001F08AF99620000201F0FEFD01232E4D3E
:101BF0005B4200202B60FEF769FE002350242B601F
:101C00000120FEF727FB00F0B5FF02F08DF92B68ED
:101C1000002B05D16420043C01F0CEFB142CEFD145
:101C20000020FEF753FE2821204802F0D1FB1420AB
:101C300001F0C2FB1D48282102F0CAFB1C4801F03C
:101C4000BCFF192001F0B8FB01F068FE002819D094
:101C50000020FEF7A3FC0821164801F0D1F902F09C
:101C600016FC03F079FB102301930E330022124976
:101C700012480093124B03F089FB124803F0BAFBA1
:101C8000FFF744FE013C002CDBD1E4E70800001024
:101C9000BE153E37E45BE173984004409C4004402D
:101CA000744004409440044094040010DE0300009B
:101CB000C073000010400440D9030000D565000047
:101CC00014060010D0050010F7B5031E019137D09F
:101CD0000278303A504242419B181A78782A13D140
:101CE0001026012501331A7800242D2A01D1013351
:101CF000013400221878002809D1002C00D052426B
:101D0000019B01201A601BE00A260025EBE7070073
:101D1000303FF9B2092903D87243BA180133E9E711
:101D200020210843002D07D00700613F052F03D86D
:101D3000120157380243F1E7024801F03EFF00204C
:101D4000FEBDC046347900000378202B00D07047D8
:101D50000130F9E703003038C2B2092A08D920203F
:101D600018430300613B5738052B01D9012040423D
:101D7000704770B50E00FFF7E7FF002504002078DC
:101D8000002802D13560200070BDFFF7E3FF002876
:101D9000F8DB2D0105430134F1E7000010B500F038
:101DA000D5FD0100014801F008FF10BD4279000097
:101DB00000B589B0684602F057F96946024801F05B
:101DC000FCFE09B000BDC04681790000F7B50E00E9
:101DD00001A91500FFF778FF002814D0019F0B49D7
:101DE000380005F097F80C006421200005F092F807
:101DF00020003170642104F0A7FF044928703800E6
:101E000004F0A2FFFEBD01204042FBE710270000C6
:101E100013B50C006B4660689A1DD91DFFF7D6FFFD
:101E20006B4698805A1C991CA068FFF7CFFF6B4641
:101E30006A4618709288044B9A4203D9694601A8F1
:101E400002F09EF913BDC0466B0700000B0007B5FA
:101E5000586801A9FFF738FF3C20019B584302F066
:101E6000A9F907BD07235843074B9C30C018831DB1
:101E70000138834201D1012070471A78013B002AC2
:101E8000F7D00020F8E7C046B80600107FB5194823
:101E900001F093FE00240326651C34421DD120006E
:101EA000FFF7E0FF002814D02800FFF7DBFF002831
:101EB0000FD0A01CFFF7D6FF00280AD0E01CFFF7C8
:101EC000D1FF002805D00434FF2CE5DD01F050FFE0
:101ED0007FBD2100084801F070FE2100684602F035
:101EE000E7FA684601F034FF044801F066FE2C0072
:101EF000EAE7C0462A7200004E79000098AC000064
:101F000070B50D00FFF720FF060004000D350E36FA
:101F100020780134FFF71EFF002807DB2870013D01
:101F2000B442F5D12000FFF70FFF70BD0020FCE7A1
:101F300070B53F4C86B02368002B07D13D4801F0B7
:101F40003CFE03F009FA012323602DE00868012B11
:101F50000FD10422384901F0AEFE002802D12368D7
:101F60000133F1E7354801F028FE03F0F5F9344973
:101F70003FE00378412B19D132490230FFF7C0FF0F
:101F80000028F2D00378422BEFD12F490230FFF71F
:101F9000B7FF0028E9D00378432BE6D12B49023064
:101FA000FFF7AEFF0028E0D006B070BD532B02D182
:101FB00027490230F4E74D2B20D126490230FFF7A4
:101FC0009FFF0028D1D003784E2BCED1224902307A
:101FD000FFF796FF0028C8D00378472BC5D1023001
:101FE00001A9FFF7C6FE019B002BBEDB154A1B496A
:101FF00053651B4801F0E1FD0023A5E701A9FFF7A8
:10200000B8FE2023057806009D43AED1300002A91A
:10201000FFF776FF019B0600E918FF2902DC02A802
:1020200002F05CFA002EA0D00135042DEED1BBE702
:10203000AC050010577900002A7200006D7900008D
:1020400086790000B8060010C6060010D4060010FD
:10205000FE060010E2060010F0060010797900007C
:102060007C79000037B54C682378002B00D137BD50
:102070002000FFF769FE01A9FFF77BFE019B04002A
:10208000002BF4D0D8B2FF2B13DD00F0C5FA019B72
:1020900005001812C0B200F0BFFA019001980028A4
:1020A00002D02900FEF712FA23785A1E9341E41851
:1020B000DAE700F0B1FA00250190EFE70123064AC4
:1020C00010B511784B401370044900D104490548FC
:1020D00001F073FD10BDC04675020010BD73000015
:1020E0008D790000917900000123064A10B511781E
:1020F0004B401370044900D10449054801F05DFDCF
:1021000010BDC04674020010BD7300008D79000040
:10211000A07900000B0007B5586801A9FFF7D4FDAE
:10212000019B002B0CDC012301939623019A9B0059
:102130005343054A01990548136001F03EFD07BD70
:102140001E2BF2DD1E23EFE730020010B0790000F5
:1021500010B50C4A1378013BDBB21370002B0AD088
:10216000012B05D10849094A094801F026FD10BD97
:102170000849094AF8E7094801F01FFDFEF7F4FA9B
:10218000F5E7C04614000010D8790000878B0000E6
:10219000DC790000D4790000F98D0000007A00009D
:1021A00070B50400002C00D170BD64250021022010
:1021B000013D00F0D9FE002DF8D1013CF2E700000E
:1021C000F0B580250F4B6D001A6804262A431A606B
:1021D00008220D4F0D491C683C401C6044B2002C85
:1021E0000CDA0C6834430C601C68013A2C43400044
:1021F000D2B21C60C0B2002AEDD1F0BD0C68B4436D
:10220000F1E7C046FC3F0150FFFEFFFFFC3F0050DE
:102210000121044A10B513688B431360FFF7D0FF08
:1022200010BDC046FC3F0250F0B583B072B601232A
:10223000843001270600194D0193B0202B6834002B
:10224000BB432B60019B843C1843FFF7B9FF2B680D
:102250000020BB432B60FFF7B3FF2B681020BB436C
:102260002B60FFF7ADFF2B68E020BB432B60FFF72F
:10227000A7FF2B683B432B6020780134FFF7A0FFBA
:10228000B442F6D1019B84342600002B02D162B601
:1022900003B0F0BD00230193CFE7C046FC3F0250DE
:1022A00010B5AC20FFF7B4FFAE20FFF7B1FFA520BB
:1022B000FFF7AEFF10BD70B50D000400012200F065
:1022C00031FE29000122200000F078FE70BD10B51B
:1022D000AF20FFF79DFFA420FFF79AFF10BD10B5B8
:1022E000AE20FFF795FF10BD10B50400F820FFF7F2
:1022F0008FFF2000FFF78CFF10BD10B50400812078
:10230000FFF786FF3F202040FFF782FF10BD00004F
:10231000202010B5064B1B781843FFF779FF0A20E1
:10232000FFF73EFF034B1878FFF7E7FF10BDC046ED
:102330001500001087040010842210B5064B0748D2
:1023400019785200002903D0054901F04CFC10BD5A
:1023500001F06AFCFBE7C046880400107E03001011
:102360007602001010B584220021024801F05CFCC6
:1023700010BDC0467E03001010B558220449054820
:1023800001F031FCB0220021034801F04DFC10BDEA
:102390007E03001076020010CE020010014B187070
:1023A0007047C04688040010002310B5074AD35672
:1023B000002B07D0013B59B21B0601D4117010BD90
:1023C000002313700248FFF72FFFF8E78604001080
:1023D0007E03001010B508210120FFF76CFF0221D9
:1023E0000020FFF768FF00210220FFF764FF0621AD
:1023F0000220FFF760FF03210800FFF75CFF0321C5
:102400000022080000F0DAFD00220621022000F080
:10241000D5FD01220621022000F0D0FDFFF78CFF40
:10242000FFF7C2FFA220FFF7F3FEA020FFF7F0FEA8
:10243000C020FFF7EDFE0020FFF756FF0A20FFF750
:10244000AFFE4020FFF7E4FE2C20FFF7E1FE322034
:10245000FFF7A6FE2E20FFF7DBFE3220FFF7A0FEDF
:102460002F20FFF7D5FE0A20FFF79AFEFFF750FF57
:10247000FFF72DFF10BD0000030083280DD80F29A2
:102480000BD88420CA085043C01807231940793359
:102490000B41024A115C0B43135470477E0300103A
:1024A000F0B5072580265B1885B0DBB2104F02908F
:1024B00003920193019B994201D305B0F0BD8422A0
:1024C000CB085343029A30009B180A002A4010415F
:1024D000039AC0B29446DA199C44634502DB013189
:1024E000C9B2E7E714780133044314700132F4E70A
:1024F0007E030010F0B587B005921E00DB788342A2
:1025000003D23778380007B0F0BDB4787268244B36
:10251000041B00209A4216D103231F005C43A41819
:10252000E318CDB20393EB19DBB2049300230193BC
:10253000049BAB42E6D0082302930023009327E0DC
:102540000233D21801301378A042F9DB5778941C7B
:10255000E6E7029B082B07D1039B9C42D2D023784D
:1025600001340193002302930122019B134206D000
:10257000059B009A28009918C9B2FFF77DFF019BBF
:102580005B100193009B01330093029B0133029384
:102590007378009A9342DCDC0135EDB2C8E7C0469F
:1025A0001B7A0000F7B505001F000C00160001F0B3
:1025B00073FB2B180193019B9D4201D0832C01D901
:1025C0002000FEBD3B00210028783200FFF792FF7B
:1025D000024B01351B68C0182418ECE718000010E6
:1025E00000210122042330B50A4C0D5D854203D140
:1025F00018011043C0B230BD013B002B04D10132A1
:102600000433092A00DD002201312829EDD1002000
:10261000F1E7C046FE8A00003C2310B504098000A3
:102620001840011F00D52831621E0020032A06D859
:10263000242904DC0423024A1B1B5218D05C10BD61
:10264000FE8A000070B505000024054B2900E05CFF
:10265000044B0134C01800F0D3FC0A2CF5D170BD36
:10266000F48A000000400440F7B50E4E3468002C98
:1026700016D11020FFF7E6FF0B4D2B786F7818006E
:10268000002239000193013400F04CFC0122390092
:10269000019800F093FC02350A2CEED1012333603F
:1026A000F7BDC0468C0400102E8B0000F8B5002545
:1026B0000B4C2678677801223900300000F032FC9C
:1026C000013500223900300000F078FC02340A2D78
:1026D000EFD10020FFF7B6FF0022024B1A60F8BDD1
:1026E0002E8B00008C04001070B50500FFF7BCFFB6
:1026F000002D09D001220721022000F013FC8021C7
:102700000F4A13688B4313600B21002000F02CFC50
:102710000124002805D00B21002000F025FC4442B4
:102720004441002D09D000220721022000F0FAFBCD
:102730008023034A11680B431360200070BDC0461C
:10274000FC3F02500023F0B58BB0069001200993A6
:102750000791FFF7C9FF0400031E01D018230124CD
:10276000089300232C4E01933778757801222900B5
:10277000380000F0D7FB00222900380000F01EFCD2
:10278000264B0293019B04330593022C1CD0029B21
:102790009B790393029B0398DB791900049300F063
:1027A000E3FB00282AD101991D4AA3008A5C08A9ED
:1027B0005A500134019B01330193029B019A023B61
:1027C0000293059B9342E0D100222900380000F0DB
:1027D000A9FB01222900380000F0F0FB114B023662
:1027E000B342C1D1002C06D00124069B089A1A607E
:1027F000079B099A1A6020000BB0F0BD049903985A
:1028000000F0B2FB0028CED00499039800F0ACFB96
:102810000028C8D0CEE7C0462E8B0000268B0000D3
:10282000FE8A0000428B0000012210B510000B212F
:1028300000F078FB00220B21012000F0BFFB0122F9
:102840000221032000F06EFB00220221032000F091
:10285000B5FB10BD37B51021244A050013680120CF
:102860008B4313608023224A9B011168214C0B4348
:1028700013600B21002200F055FB00220B210120E8
:1028800000F09CFB9F211C4B1A688A431A601A684F
:102890001A491A601A4B186804F056FA030280208D
:1028A000184320602A000320022100F087FB0A2041
:1028B000002D00D0012000F07FFDFF22236893430C
:1028C000236022680F4B13430F4A23601368019360
:1028D000019B002BFADA23680C4A13402360FFF7B0
:1028E000A3FF01980004800D3EBDC046388204401D
:1028F0008080044000C001409840044000093D0031
:1029000098040010800000012CC00140FFFFFFF878
:1029100010B50D4C2068002814DA00202060FFF765
:1029200099FF0A280BDC0120FFF794FFE0234138D0
:10293000FF385B00984202D8C03BFF3B2360FFF7A3
:1029400073FF206810BDC0461C00001010B5FFF7D3
:10295000DFFF002801D1002010BD0020FFF77AFF23
:102960000120FFF777FF011EF5D0024804F0ECF9D3
:10297000F2E7C0462D47130010B5FFF7C9FF002846
:1029800009D0FFF7E3FF00210300034AC00F9A427A
:102990004841024B186010BD34080000900400103C
:1029A0000222074B10B51A60064BA0321960064B85
:1029B0001A70013258709A7000F0F0FD10BDC046D8
:1029C000FC050010E8050010D40500100022064B9D
:1029D000023110B51960054B1A60054BA2321A700E
:1029E000587000F0DBFD10BDFC050010E80500107C
:1029F000D405001070B505000E0003243100280036
:102A0000FFF7CEFF0223FF33984202D0013C002C97
:102A1000F4D170BD70B505000E000324310028000C
:102A2000FFF7D4FF0223FF33984202D0013C002C71
:102A3000F4D170BD0A4B10B51B68002B0ED0094CA9
:102A4000A31CA270140A5C70140C120EDA709C7035
:102A5000FFF7E0FF831EFF3B5A425341180010BDB1
:102A600094040010D405001070B50E4C2468002C9E
:102A700015D00D4C160AA270E670160C120E62717B
:102A8000A371A21D26711C0A54701C0C1B0E94709D
:102A9000D370FFF7BFFF841EFF3C63425C41200000
:102AA00070BDC04694040010D4050010064B10B54C
:102AB0001B68002B05D0FFF79DFF831EFF3B5A428A
:102AC0005341180010BDC04694040010064B10B5C9
:102AD0001868002807D007210220FFF78BFF023873
:102AE000FF384342584110BD940400100E4B70B59E
:102AF00004001868002813D0A11E062911D8072544
:102B00006D1A072D04D009482A00091801F06BF846
:102B10002900E0B2FFF77EFF0238FF3843425841F8
:102B200070BD01204042FBE794040010D605001060
:102B3000012110B50800FFF75DFF0223FF33984223
:102B40000FD10120084B1860084B1C78230706D0D2
:102B50000323074A234001009370FFF75BFF200027
:102B600010BD01246442FAE794040010EC05001043
:102B7000D405001010B5FFF7DBFF01210220FFF79D
:102B800039FF0223FF3398420FD1084B1B787F2B6C
:102B900006D9842207210220054B5204FFF764FF67
:102BA00004210920034AFFF745FF10BDEC05001082
:102BB000020114008080808010B5002848D0802158
:102BC000254A13688B431360012324490A681A427B
:102BD000FCD00322224B1A6001230021214A1360FA
:102BE0001160136011681942FCD01F4A1F4913601D
:102BF00080230C685B0223430B60002804D18023F0
:102C000015490C6823430B60194B196881421ED08B
:102C10001860431E9841174B40421840164B1168EC
:102C2000C01804F007F8FA21144B8900186004005A
:102C300004F08AF81E23C8214343114A2000136080
:102C4000490104F081F80F4B186001F051F810BDF4
:102C5000034B1860C0E7C046388204400C80044033
:102C60007080044074800440788004408080044078
:102C70002000001000512502001BB700980400102E
:102C8000A00400109C04001010B500F03DF9134A98
:102C9000002113681B0B1B031360114A13681B0BE5
:102CA0001B0313600F4A13681B0B1B0313600E4AB0
:102CB00013681B0B1B03136001220C4B19600C4B98
:102CC0001A6019601A6019681142FCD02322094B5E
:102CD00000201A60FFF770FF10BDC0460080005052
:102CE000008001500080025000800350408004406A
:102CF0004480044008800440014B024A1A60FEE709
:102D00000CED00E00400FA0570B500250B490C48F5
:102D100000F053FF0B4E300000F04FFF0A4CE2680A
:102D2000216833000948013500F047FF14340C2DA9
:102D3000F5D1074800F041FF70BDC0462A7200007F
:102D4000428B0000858B0000C08C0000548B00007B
:102D50005F8B0000F0B500253D4F04003B68280064
:102D60008BB0AB425ED03B4B02941B6802A99B68C0
:102D7000013098473B68002B02D1374800F01DFF17
:102D80000BB0F0BD01342378202BFBD0002B2FD0CB
:102D9000431C0193800002ABC450FF2D06D1019B60
:102DA0001800022B45D1002526E01C002278002ABD
:102DB00005D0631C202AF8D1002222701C00019B40
:102DC000012B2ED10C26234D244B2B602B6802980F
:102DD000196800F080FF2B68002821D01433013ED1
:102DE0002B60002EF2D131003000FFF78DFFC4E7D9
:102DF0000028BFD002281AD11949039800F06BFFB0
:102E000000280BD1134C17482368D96800F0D5FE71
:102E100023681548196900F0D0FEABE7022006E0F0
:102E20001D7901982378002BE2D00828ABD1854288
:102E3000E8D2084CC0B2236802A99B689847226870
:102E40000A4B92689A4295D00322094B1A7091E777
:102E5000AC050010A4040010888B0000C08C00009A
:102E60005B720000818B000081790000512100001D
:102E70001400001070B50400154D0D281BD00CD89F
:102E800008280CD00A2816D02100124800F095FE20
:102E90002B685A1C2A601C7018E07F28F4D10E4B56
:102EA0002A689A4212D921000A4800F086FE2B684F
:102EB000013B2B600AE000232A680848137000F0E9
:102EC0007CFE054C2000FFF745FF2C6070BDC0461E
:102ED000A8050010948B0000A8040010858B00004A
:102EE00010B500F01BFD002800D110BD00F0F4FC6F
:102EF000FFF7C0FFF5E70000014B024A1A60704778
:102F0000A8050010A80400104023044A11680B43D0
:102F100013600122024B1A707047C0468080044043
:102F2000B00500100E4B70B51B7804000E001500A4
:102F3000002B01D1FFF7E8FF631E022B0AD8094BD3
:102F40002004C01801230268B340012D04D11343AB
:102F5000036070BD0348F5E79A430260F9E7C04695
:102F6000B0050010008000500F4B70B51B780500B5
:102F70000C00002B01D1FFF7C7FF0020032D0BD859
:102F80002800012303F038FE02090B0D074AA34075
:102F900010681840431E984170BD054AF7E7054A7E
:102FA000F5E7054AF3E7C046B0050010FC3F0050C6
:102FB000FC3F0150FC3F0250FC3F03500E4B70B5EC
:102FC0001B7804000E001500002B01D1FFF79CFFB9
:102FD000631E022B0AD8094B2004C0180123026883
:102FE000B340012D04D11343036070BD0348F5E7DE
:102FF0009A430260F9E7C046B0050010FC3F00505C
:10300000084B70B51B7804000D00002B01D1FFF7B1
:103010007BFF182223689343236021680D432560BA
:1030200070BDC046B00500103F224021044B1A601D
:10303000044B3E3A1A60044A13688B43136070478E
:1030400024800440D8800440388204404021044A4F
:1030500010B513688B431360FFF7E6FF10BDC04641
:103060003882044009490A4A0B681A4080235B00F1
:1030700013430B600421074A13688B431360064B0C
:103080001A68064B1A6030BF7047C0460080034084
:10309000FFF7FFFF10ED00E0388204403482044067
:1030A00010B500F041FAFFF701FB00210948FFF7D6
:1030B000A7FF00210848FFF7A3FF00210748FFF7FB
:1030C0009FFF00210648FFF79BFF00210548FFF7FF
:1030D00097FF10BD0840044000400440AC4004404D
:1030E000144004401C40044010B50120FDF7B2F824
:1030F00010BD00008022124B10B5DA679218DA6713
:103100008022D200DA6780225201DA67802212011F
:10311000DA6780229200DA6700230121094A4942D6
:103120001360094A1160094A1360094A1360094A89
:1031300001331360084A1360FFF7D6FF10BDC04685
:1031400004E100E0048204400882044004C000401E
:103150003CC0004000C0004000400140064A10B59D
:10316000136801331360054B1868FFF725FDFFF75F
:10317000C1FFC046C04610BDB805001020000010B9
:10318000F0B585B00C00019072B6FFF789FF554B82
:10319000554D1A68554B1A60019B5A1E93413F22A8
:1031A0005B429343524A9B18524A13600423524A8B
:1031B00011680B43136000232B60A3071AD04F4AFA
:1031C0004F4913680B40136029684E4BA20700D487
:1031D00082E0EC2252010A432A6080221A6092188F
:1031E0001A608022D2001A60802252011A60802266
:1031F00012011A60019B002B53D00024424B434F15
:10320000434E3C601C60434B21001C60424B30002D
:103210001C60FFF7F5FE220009212000FFF782FE67
:10322000220009212000FFF7C9FE80213B4A3C48CB
:1032300013680B4313600722336876399343336076
:103240003368053A13433360019B584303F0F2FCA3
:103250000322344B34491860344B1C60344B1A60E1
:10326000344B1A680A4080211A601A680A431A60AF
:103270008023244A21499B0013600A681A430A608C
:103280002A68022113432B6001232B4A13602B4A27
:1032900011602B4A13601460136011681942FCD04E
:1032A0003B6001220021274B52421A60264A1368D4
:1032B0000393264B196062B630BFC046039912686B
:1032C000914207D101221A60214B1868FFF774FC64
:1032D000FFF710FF05B0F0BD802212010A432A60FB
:1032E00085E7C046388204400482044034820440AA
:1032F000FF1800003082044010ED00E0008204401E
:103300007FE2FFFF00E100E00400014004C0004054
:103310006440044004400140048001408080044037
:10332000841E000018C000400FF0FFFF08C00040DE
:1033300014C000403CC000407880044070800440CD
:103340007480044008820440B8050010B4050010E1
:103350002000001010B5FFF713FF10BD074B1A68CF
:10336000013203D106490A6801320A601A68013243
:103370001A60044A1368013313607047C8050010CF
:10338000C4050010C005001080235B0498420AD2D7
:103390000023054A01381360044A1060044A136090
:1033A0000722044B1A607047C805001014E000E0C3
:1033B00018E000E010E000E00B4A1368002800D19C
:1033C0000130C143994209D2591C08181168994229
:1033D00000D2704711688842FCD8F7E71168C91A13
:1033E0008142FBD3F5E7C046C8050010014B1868C1
:1033F0007047C046C80500100122034B1A60034AFB
:10340000136801331360704700C00040CC05001002
:103410000122034B1A60034A13680133136070479B
:1034200000000140D0050010002803D10122044B08
:103430001A6070470128FCD1024B1860F9E7C046BA
:1034400004C0004004000140002802D1044B186071
:1034500070470128FCD10022024B1A60F8E7C046F1
:1034600004C0004004000140002805D1044A0223A2
:1034700011680B43136070470128FCD1014AF6E73D
:1034800004C000400400014010B5002900D11449D7
:10349000002810D18023134A1468234313600322A9
:1034A000114B1860114B1960114B1A608022114B9F
:1034B00052021A6010BD0128FCD18023094A5B002A
:1034C00010680343136000220B4B1A600B4B03324E
:1034D00019600B4B1A608022064B9202E9E7C04646
:1034E000FFFF000080800440CC05001018C00040A1
:1034F00014C0004000E100E0D005001018000140B9
:1035000014000140802210210820064BD2051160D2
:10351000186080235B011068084202D0013B002B39
:10352000F9D17047180000408022164B120210B5E6
:10353000DA676C22144B15481A60154B1968014064
:1035400019601A6804211A60124B1A6802401A6046
:103550001A6800201A600122FFF7E4FC012204210E
:103560000020FFF72BFD012205210020FFF7DAFCE8
:10357000012205210020FFF721FD0022064B1A60E1
:1035800010BDC04604E100E018000040F8FCFFFF59
:10359000304004403440044004800440F8B5002327
:1035A000164A174C202123601360164A13608022AC
:1035B000D2051160144A2168012907D0934203D132
:1035C000FFF7A0FF0020F8BD0133F4E79342F7D0E6
:1035D00000250E4F3E68013E2368FF2B01D920686D
:1035E000F1E73B68B34204D03E68FFF7FFFE0A30C4
:1035F0000500FFF7FBFEA842EED1E1E70006001050
:10360000E405001004060010FF0F0000080600107B
:103610000122034B1A60034A136801331360704799
:10362000004001401406001070B50124164B174AE3
:103630001C6013681B191360154B1A68002A13D0FD
:103640001A68144D013A1A601E68002E0DD0210030
:1036500020002A68FFF7B2FC2B680221E31A2B60D6
:1036600020002A68FFF7AAFC70BD1B6821002B60B0
:1036700020002A68FFF7A2FC022120002A68FFF739
:103680009DFC054B1E60EFE700800140180600100E
:103690000C0600101006001004800140002803D121
:1036A0000122044B1A6070470128FCD1024B1860BC
:1036B000F9E7C0460440014004800140002802D1DF
:1036C000044B186070470128FCD10022024B1A609D
:1036D000F8E7C0460440014004800140002805D1BD
:1036E000044A022311680B43136070470128FCD180
:1036F000014AF6E7044001400480014010B500286B
:1037000011D18023124A9B001468234313600322C3
:10371000104B1860104B1960104B1A608022104B30
:10372000D2021A6010BD0128FCD18023084ADB00B8
:1037300010680343136000220A4B1A600A4B0332DD
:1037400019600A4B1A608022054B1203E9E7C04654
:1037500080800440140600101840014014400140CD
:1037600000E100E0180600101880014014800140BC
:103770000E22174B10B51B681340062B12D1154BA8
:1037800090321B68134205D0134ADBB25360134BCF
:103790001B6810BDDB07FCD5104B1868C0B200F0E9
:1037A000ACF8F6E7042BF7D00C2B05D10A4AF4331A
:1037B00051680B435360ECE7022BEAD1054B1A68C2
:1037C000054B920602D500229A60E2E70122FBE750
:1037D00008800040148000401C060010008000405B
:1037E000004870471C060010F7B58022002107250D
:1037F0002A4B2B4C9203070001912000DA6790229C
:1038000000F012FA019B274EA360274B1A68AA43C7
:103810001A600122196811431960244B1968A943E1
:103820001960196811431960802321495B010868F8
:1038300003430B601F4B1A60823232601E4A1268CB
:1038400019681E4B1868504303F0F4F93900000959
:1038500003F0F0F910221A4B1A491A60030A0B60A0
:103860000323194FC0B2386060203360174B1D60CE
:10387000174B1A6801921A680240602AFBD15F3A1E
:103880001868104207D122708022124B92031A60EE
:1038900005230B60F7BD38680190F1E704E100E013
:1038A0001C0600100C800040A4400440A8400440C6
:1038B0008080044098800440788004409804001080
:1038C00028800040048000400080004008800040C4
:1038D0001480004000E100E010B5FFF781FF020016
:1038E000837BC318D87B937B0133DBB293735BB2CA
:1038F000002B01DA0023937310BD10B50400FFF70D
:103900006FFF437BC318DC73437B0133DBB243732C
:103910005BB2002B01DA0023437310BD10B5FFF733
:103920005FFF0300807B5B7BC01A431E9841C0B2DF
:1039300010BD70B504001D0000202E5C2318002E61
:1039400009D1121AD518EC1A002C07DCD343DB1767
:103950001A40101870BD26540130EEE7197001337B
:10396000F1E7F8B5541E0F001E000500230001000A
:10397000092E16D90A21300003F05CF92200030059
:1039800039002800FFF7EDFF04002D1830000A2150
:1039900003F0D6F930312970601CF8BD0F70013B7F
:1039A0000131002BFADC0020824200DD20002D18BE
:1039B000002A00DC0122541EE8E7F7B50E00D917F3
:1039C0005F18040001934F40551E092F17D90A2193
:1039D000380003F02FF9019A0300002A00DA43426D
:1039E0002A0020003100FFF7E8FF05002418380006
:1039F0000A2103F0A5F93031681C2170FEBD019B3E
:103A0000002B00DA951E23006119CA1A002A0CDC6B
:103A1000E843019AC017054064196B1C002AE6DAD6
:103A20002D221D0022700134E1E71E700133ECE706
:103A3000F7B51E00089B1400013A1F09050013008A
:103A4000002F11D033000097FFF7F2FF2D180F233E
:103A5000089F1F40FAB2092F12D830322A70013065
:103A6000FEBD0170013B0130002BFADC00208442D6
:103A700000DD10002D18201E00DC01200138E6E7D3
:103A8000002E01D03732E9E75732E7E7F0B50500FD
:103A90000F001C0085B0002801D000230370002611
:103AA0001378002B00D16DE0B74204D80023013D0C
:103AB0002B70013E32E0252B04D001322B700136F1
:103AC0000135EDE75178252902D129700232F6E758
:103AD000931C0393302902D02021531C0393039B92
:103AE0001B782D3B5A425341039AD318002203936B
:103AF000039B1B7818003038092812D99019B84256
:103B000001D9BA1BD2B2692B1FD013D8632B35D081
:103B1000642B1AD0582B2DD001267642300005B0E8
:103B2000F0BD0A2042439A18039B303A0133D2B2C7
:103B30000393DDE7752B11D0782B14D0732BEBD1C9
:103B4000280008CCFFF7F5FE03E0280008CCFFF7BB
:103B500034FF039A2D1801323618A1E7280008CC4B
:103B6000FFF7FFFEF5E708CC009300232800FFF7DE
:103B70005FFFEEE708CC00930123F7E708CC0120B4
:103B80002B70E6E7B74200D890E72B70C6E710B578
:103B900013000A006421FFF779FF10BD00B59BB048
:103BA0000A00010001A8FFF7F2FF632800DDFEE72D
:103BB00001A800F0C3F81BB000BD0FB407B504A9FD
:103BC00001C90191FFF7EAFF03B008BC04B0184730
:103BD0000EB403B503AA02CA0192FFF7D8FF02B0E0
:103BE00008BC03B0184770B506000E430325340027
:103BF00003002C402E420FD1AA420DD90B5903517C
:103C00000434131B032BF9D80324131F9B0801331F
:103C10009B00C9182240C3180024A24200D170BDE5
:103C20000D5D1D550134F8E770B5830704D003001E
:103C30009A189A4217D170BD0300032AF8D90C04D0
:103C40000B0623430B430C0223430400861808C4CD
:103C5000351B032DFBD80324131F9B0801339B0046
:103C6000C3182240E4E719700133E2E710B581423E
:103C700008D20139431E002A00D110BD8C5C9C542F
:103C8000013AF8E78142F8D9002302E0CC5CC45441
:103C900001339A42FAD1F0E7030000201A5C002AAF
:103CA00000D170470130F9E70023CA5CC2540133E8
:103CB000002AFAD1704770B5002304009A4201D15E
:103CC000002007E0E55CCE5CA81BB54202D10133C1
:103CD000002DF3D170BD0200002310B5D05CCC5C88
:103CE000A04201D0001B02E001330028F6D110BD34
:103CF000FA21094B10B51868890003F025F8FFF781
:103D000043FB96200002FFF76FFD0120FCF7A2FAAB
:103D1000FEF730FF10BDC0469804001010B5FEF746
:103D2000B3FFFFF7F1F8FFF791F9FEF753FBFEF74A
:103D300003FBFFF7DDFFFFF7DFF810BD10B5040050
:103D40002078002800D110BD0134FCF7D9FAF7E73C
:103D500070B50500441E0D35A54200D170BD29780F
:103D60000248FFF72AFF013DF6E7C0465F730000F7
:103D700070B51748FFF721FF164D2800FFF7E8FF41
:103D8000154C42212000FFF718FF1448FFF7E0FF11
:103D900043212000FFF711FF1148FFF7D9FF114819
:103DA000FFF70BFF1048FFF7D3FF1048FFF705FFA1
:103DB0000F48FFF7CDFF4E212000FFF7FEFE0D4814
:103DC000FFF7C6FF696D0C48FFF7F7FE70BDC046F0
:103DD000B08D0000B8060010B68D0000C6060010B9
:103DE000D4060010BD8D0000FE060010C38D00003B
:103DF000E2060010F0060010C98D00000A2302112F
:103E000053430F2210401818704770B50A2105005F
:103E100002F09AFF0A210401280003F07BF8200039
:103E2000084370BDC12210B5520002210E20FEF7DA
:103E300001FE0122014B5A7110BDC046AE060010B2
:103E400010B5084C6379002B01D1FFF7EBFFA27985
:103E50002379520001211A430C2308001A43FEF76C
:103E6000E9FD10BDAE06001010B5074C2379002BFC
:103E700008D16379002B01D1FFF7D4FF012323710F
:103E8000FFF7DEFF10BDC046AE06001010B5054BB3
:103E90001A79002A05D000221A711A72DA70FFF717
:103EA000CFFF10BDAE06001010B501210220FEF7B5
:103EB000FDFD064B040018787F231840FFF79EFF96
:103EC000034B5870DC71200010BDC046EC0500109B
:103ED000AE0600100122014B9A707047AE0600102A
:103EE0000022024B9A701A727047C046AE0600104C
:103EF00010B5FFF7D9FF094B09499A78002A03D07A
:103F00001A7A012A02D801321A7202E00868054AB8
:103F100010600022DA700A6010BDC046AE060010C4
:103F2000C0050010BC05001010B5FEF701FE0C2204
:103F300003001340104203D0024A11780B43137060
:103F400010BDC046AE06001010B5FFF7EDFF044CE3
:103F500023785B0701D5FFF7CBFF0023237010BD4B
:103F6000AE06001010B50020FEF7BEFB002801D001
:103F7000FFF7EAFF10BD0000002310B5044CE37109
:103F8000FFF7F0FFE379002B01D1FFF78DFF10BDA4
:103F9000AE06001010B50921084803F0EFF8FA2228
:103FA000074BD2001A80FFF7E7FF0022054B1A608B
:103FB000FA22054B92001A6010BDC046AE060010F2
:103FC000AC060010C0050010BC05001010B5FFF7CE
:103FD000C9FF002010BD704710B5FFF757FF10BD97
:103FE00070B51D4C0D0061782378A2780902194341
:103FF000E378120411431B06184A0B4313401A0AB4
:10400000237062701A0C1B0EE37063792179A27021
:104010001B02134A0B43134023711B0A06006371F2
:10402000A079FFF7EBFE0F4B1B881B1833806079DC
:10403000FFF7E4FEB070E078FFF7E0FEF070A078E4
:10404000FFF7DCFE28706078FFF7D8FE68702078F4
:10405000FFF7D4FEA87070BDEC0500107F7F3F3FD6
:10406000071F0000AC060010F0B58DB00400FEF78D
:104070002DFD002805D120001249FFF7A9FD0DB044
:10408000F0BD0AAE0BAD29003000FFF7A9FF338861
:104090000793F378B77808932B7809930A4B6E78D7
:1040A0001879AD7800F0D2F8099B04900193089B31
:1040B00020000093079A3B00044903950296FFF7FE
:1040C00087FDDCE7D58D0000EC050010DA8D0000DF
:1040D00070B505000E001400FEF7F8FC00280AD0A9
:1040E00028003100FFF77CFF201E03D00020034B87
:1040F0001B79236070BD01204042FBE7EC050010F6
:10410000F7B504880E000500642120000092019399
:1041100002F016FE114B8FB2E41B1C80B078FFF743
:1041200074FE0F4CA0707078FFF76FFEE07030786F
:10413000FFF76BFE2071E878FFF767FE009B607168
:10414000A371A878FFF761FEE0713800FFF75DFE0C
:1041500020720198FEF7CAFCFEBDC046AC060010F6
:10416000D405001010B50223FFF7CAFF10BD431E8F
:10417000984110B5420101210020FEF75BFC10BD03
:1041800070B5040001200D00FFF7F1FF200000F0E2
:1041900085F8072102F0BEFE20000A002900FFF783
:1041A000E1FF96204000FFF707F90020FFF7DFFF4F
:1041B00070BD000073B50400FFF776FE002801D142
:1041C000002076BD1D4D6E780A20FFF7F5F8FFF749
:1041D0006BFE0028F4D06B78B342F5D0FEF776FC86
:1041E0000028EDD001A96846FFF7FAFE684600F006
:1041F00055F8050001A800F031F8114B04199C4254
:104200000DD90122E3171343ED186946280000F089
:1042100077F80C4AE31713400B4A9B18E418200068
:1042200001A900F025F82800072102F073FE684676
:104230000A0001A9FFF796FFC3E7C046AE060010CB
:104240007F51010000A3020080AEFEFF072318404B
:10425000014B8000C0587047188E00003C230200BC
:1042600000785178584340184343907818187047A5
:1042700070B50C003C21050002F04CFE2800A17036
:104280003C2102F061FD3C2102F044FE6170E1211D
:104290002800090102F058FD207070BD70B596220B
:1042A00083780688050000205201B618010002221A
:1042B0009A424141761A022B00D80C30C01899233B
:1042C000033858436E240521023002F03DFD64217D
:1042D000FF3474430419B01024184942300002F02E
:1042E00033FDC82124184900300002F02DFD034B96
:1042F0002018EC78C018001970BDC046D382FFFFAB
:10430000F8B5214B050080000E00C0181F4902F0CF
:104310001BFD032703007B43D8173840C0188010CB
:104320001B4B2D18AD00ED1828001A4902F0F2FDC4
:10433000CC173C4064180237A4107C4302342000A0
:10434000992102F0E7FD0800390002F0FDFC013080
:10435000F0709921200002F0F7FC0C21023002F0ED
:10436000D9FD0131C8B20E21B070081A023902F02D
:10437000EBFC08490400280002F0E6FC064BC018DC
:1043800024183480F8BDC046652F0400B13A0200FD
:104390004F150000B505000094EDFFFF012210B598
:1043A00011001000FEF70AFE012202211000FEF7A4
:1043B00005FE012100220800FEF7B4FD00220221C3
:1043C0000120FEF7AFFD0120FFF778F910BD0000D6
:1043D00070B50D00072101240600174B20001A6854
:1043E0008A431A601A6822431A60144B1A688A4377
:1043F0001A601A68210022431A602200FEF792FD1B
:10440000220002212000FEF78DFD0D4B31001868BF
:1044100002F09AFC01002000FFF770F92000FFF77E
:104420005DF9084E20003560FFF738F93368002B3E
:10443000FCD1FFF7B3FF70BD7C40044080400440D6
:10444000980400100C0600100300F8200A00C000B9
:10445000890101405005800E0143F820000202400E
:1044600011430A22514330B5CC101A191000EB3019
:1044700055780078EA32684012781B5D00021043DC
:1044800058400723194008418005800D30BD704712
:10449000C023010010B55B01984201DB024BC1183B
:1044A0000248FFF7D1FF10BD00F8FFFF4E8D00005E
:1044B0000723020010B50F245943074B9C31C9183C
:1044C0000E320B78234003700B7801311B094370C7
:1044D00002309042F5D110BDB8060010072302004B
:1044E000594310B5064B9C31C9180E3243780478F5
:1044F0001B01234302300B7001318242F6D110BD03
:10450000B806001070B5B64D1726EB6E86B05A1E71
:1045100093416E443370B34BEA58D006400F0138D4
:10452000062808D802F068FB443104363C3F4200BC
:104530000D23002404E06B6E16339B005C592300AE
:1045400050111F283BD802F06BFB35003F004400A0
:1045500048004E00560059005F0063006900780073
:10456000830090009F00AC00B700C400D100DF00C2
:10457000EC00FD00FB000A011101160123012E01D0
:10458000330137013D01410145016B6E16339B003C
:10459000EB58CEE7AC6DEB6D9C42D1DD0D23CFE740
:1045A00002231C00CCE70C230324C9E70D23F8E702
:1045B0000223BEE7191B0131281902F0DFFD01209B
:1045C0003378EB6606B070BD191B8748013120189F
:1045D000F3E7191B85480131F9E7220082492800D9
:1045E00001F0B1F9EBE71A1B7F48013229192018B5
:1045F000FFF7F9FAE3E722007C49F0E77A491A1B52
:104600007A4801326118F2E7220078497648E7E7F4
:1046100076491A1B013261182819E9E7296E0A2226
:10462000002900D106320093230002926E4A0196BF
:104630002900280001F091F9C1E7296E0A2200291A
:1046400000D1063202920093684A23000196EFE7F8
:104650000122296E32700932002900D106320292FD
:104660000093002223000196E2E7296E0A22002926
:1046700000D106320093230002925B4A0196290082
:10468000280001F095F99AE70122296E327009326B
:10469000002900D1063202920093002223000196E5
:1046A000EDE7296E0A22002900D10632029200931A
:1046B0004E4A23000196E2E7296E0A22002900D122
:1046C00006324A480292009302002300019601003C
:1046D000B0E7296E0A22002900D10632434802922F
:1046E00000930200230029000196A3E70122296E0E
:1046F00032700932002900D1063202920093002262
:1047000023003A480196E2E7296E0A22002900D1E7
:1047100006323648029200930200230029000196D7
:10472000AFE70122296E32700932002900D106322A
:104730002E48029200930022230001000196A0E778
:1047400001223270296E0A22002900D10632274840
:1047500002920093020023000021019691E72200BB
:1047600000212148009601F085F928E72200002168
:104770001E480096F7E7296E0A22002900D106326A
:10478000009323000292194A01962900002078E73D
:10479000296E0A22002900D1063202920093124AA1
:1047A00023000196F1E72200002100962800DAE7B5
:1047B00022000E490096F9E71A002100280001F0B6
:1047C00070F9FCE61A0021000748F8E71A002100FA
:1047D0000648F4E71A002100280001F073F9EEE61C
:1047E000B8060010C4070000C6060010D40600106A
:1047F000064B10B519001A1DD46F0831CC67D96F5C
:10480000D1679A6F9867DA6710BDC046B806001086
:10481000064BDA6F986F9A671A1DD16F0833596784
:10482000D96FD1670022DA677047C046B80600101A
:10483000F8B5134D2F008C373B68581CFFF728FE46
:10484000F923DB00E8500123AA6E040003409A42DA
:1048500013D10C4BEE58830703D438680230FFF7AE
:10486000C7FFFF202B000122A40100020440B61064
:104870008C3334431C60044BEA500220F8BDC04620
:10488000B8060010C4070000AC0700000D4B0E492D
:104890000120CA5810B5D3059B0E94050ED5403B98
:1048A0008C6E92100240944206D10A008C32146839
:1048B000E3181360054BC850012010BD002BEFD149
:1048C0000300EDE7C4070000B8060010AC070000C5
:1048D00010B5084B5A1CD07F9A1CD27F00011202DF
:1048E000104303331A7FDB7F10431B031843FFF78A
:1048F0007FFF10BDB806001010B5FFF789FF0F2429
:104900000323044A01002140D15401330011072B35
:10491000F8D110BDD406001010B5FFF779FF044B95
:1049200001211A008C321060024A995010BDC04615
:10493000B8060010AC07000010B5064CA36E002BA3
:1049400007D0FFF765FF230001228C331860024B6C
:10495000E25010BDB8060010AC07000010B5064CC0
:10496000A36E002B07D1FFF753FF230001228C33E6
:104970001860024BE25010BDB8060010AC070000F2
:104980000121054B054A10B5D150054B1B68002B82
:1049900000D0984710BDC046BC070000B806001004
:1049A0008C0E00100020144B144A70B5985004323D
:1049B0009A5882421AD0F622D2009958814214DDC8
:1049C000012909D1F721C9005C58844204D058500C
:1049D0000A210B4D99505C51F621C9005A58032AFF
:1049E00001DD0120D866013A5A5070BD054B1B68A5
:1049F000002BFAD09847F8E7B8060010BC07000073
:104A0000B40700008C0E0010F822094BD2009A580F
:104A1000002A04D0F622D2009A58002A07DD0F217E
:104A2000044A9A580133114012119977DA77704786
:104A3000B8060010B4070000044A537F917F1B01A1
:104A400009020B43117F0B4353677047B8060010F0
:104A50000B00093B30B5012B0BD80023074AD55C6E
:104A6000C45CA54206D0064A064B0839D05801431B
:104A7000D15030BD01330E2BF1D1FAE7D40600102E
:104A8000B8060010A407000010B508290FD0192996
:104A900008D1082342781A4205D0002202704370E0
:104AA000FFF71CFD10BD0F230370083BF7E7020062
:104AB000030000240E321C7001339342FBD1EFE758
:104AC00030B5114B85B05C6F002802D00F229443A3
:104AD00004430E4D5C67FF2C05DD0E21280002F01B
:104AE0004DFB05B030BD21006846FFF7E1FC210019
:104AF0006846FFF7C9FF00236A46D25CEA540133D7
:104B00000E2BF9D1EDE7C046B8060010D406001010
:104B10001FB50F22104B5C6F944304435C67082C55
:104B200018D0FF2C16DC21006846FFF7C1FC2100DD
:104B30006846FFF78DFF002308496846CA5CC254E7
:104B400001330E2BF9D12100FFF79EFF21006846AB
:104B5000FFF7C4FC1FBDC046B8060010D406001005
:104B60001FB50E4C616F082917D0FF2915DC684668
:104B7000FFF79EFC616F6846FFF76AFF0023084954
:104B80006846CA5CC25401330E2BF9D1616FFFF73E
:104B90007BFF6846616FFFF7A1FC1FBDB8060010E0
:104BA000D406001010B50D4C631CD87FA31CDB7F0E
:104BB00000011B021843E37F1843E31CDB7F1B0348
:104BC0001843FFF765FC0F220300134023770311FE
:104BD000134000126377A07710BDC046B8060010DE
:104BE000024A536E16339B00D0507047B80600102F
:104BF00004494A6E1632920053581B1A5A425341C6
:104C0000CB667047B8060010054A536E16339B00FA
:104C10009958013901D4995070470D21FBE7C046DE
:104C2000B8060010064A536E16339B009958481C6C
:104C30000D2901D09850704700219950FBE7C046DC
:104C4000B80600100F4B5A6E16329200D058191841
:104C50000A7F0C2804DC497F09010A435A65704722
:104C6000F5200949120159588000814205D00748B2
:104C70000140B7208000814202D1596D0911ECE753
:104C8000197FEAE7B8060010CC070000FFFEFFFF1F
:104C9000224B30B55A6E16329200D2580C2A05D1EA
:104CA000F5211F4889001858884204D0FA21C9000C
:104CB000595800290DD00F20596D9A1808400C1131
:104CC00050771477FF220901114021431877596565
:104CD00030BD0F25586D041105400C2A03DC9B18CC
:104CE0001D775C77F4E70E4A9958F52292009142BD
:104CF00005D00C4A1140B7229200914208D11A0007
:104D0000FF212932157002010A4022435A65DFE76C
:104D10001A00293214701D77DAE7C046B806001071
:104D2000CC070000FFFEFFFF0F21254B70B55A6E28
:104D3000586D16329200D258014000110C2A05D14C
:104D4000F524204DA4005D59A54204D0FA24E400C6
:104D50001C59002C0CD0551C5D192C7F9A18167FFD
:104D6000240134435C651C7F2C77107719770CE0A5
:104D7000C9B20C2A0ADC551C5D192C7F9A18167FC3
:104D80002401344328775C65117770BD1D00F5263A
:104D90000C4A29359C582A78B6001201B44205D035
:104DA000094E3440B726B600B44204D102435A65D6
:104DB00029331970E9E71C7F287022435A65D5E72B
:104DC000B8060010CC070000FFFEFFFF10B50E2252
:104DD00002490348FEF707FF10BDC046D406001085
:104DE000F006001010B50E2202490348FEF7FBFE44
:104DF00010BDC046F0060010D406001010B50D23FB
:104E000000220249024800F09EFD10BDF00600108D
:104E1000D406001010B50E2202490348FEF7E3FE47
:104E200010BDC046D4060010E206001010B50E22D8
:104E300002490348FEF7D7FE10BDC046E206001047
:104E4000D406001010B50D2300220249024800F0DC
:104E50007AFD10BDE2060010D4060010024B1818AF
:104E600046300278DA667047B8060010044B00221C
:104E700019009A6408314C33CA871A807047C046BB
:104E8000B8060010C21C431E002010B504499A4207
:104E900000D110BD8C5C40002043013AF7E7C046CA
:104EA000FE06001030B50124054A0B1D994200D1C1
:104EB00030BD05002540555440100131F6E7C0468D
:104EC000FE06001070B50020FFF7DCFF0500084C5F
:104ED0000021207FFFF7E6FF25770420FFF7D2FFB0
:104EE00005000421607FFFF7DDFF657770BDC046D8
:104EF000B806001010B50020FFF7C4FF034C207760
:104F00000420FFF7BFFF607710BDC046B806001051
:104F100010B5054C0021207FFFF7C4FF0421607FFE
:104F2000FFF7C0FF10BDC046B806001010B50A4C10
:104F300023008C3318680130FFF7AAFAF923DB004D
:104F40000F22E05003001340237703111340001297
:104F50006377A07710BDC046B806001010B50E21CB
:104F6000054802F00BF90E21044802F007F90E2162
:104F7000034802F003F910BDB8060010C606001081
:104F8000D40600100022054B197F18780132014326
:104F9000197701330E2AF7D17047C046B8060010C2
:104FA0000022054B187F197801320140197701332F
:104FB0000E2AF7D17047C046B80600101FB500236F
:104FC0000A4A6C461118097F013019550D2800DD79
:104FD000002001330E2BF4D10023054A6946C95C39
:104FE000D15401330E2BF9D11FBDC046B8060010B5
:104FF000D4060010074A10B5536E16339B0099581B
:105000004C1E51189C500877002C01DA0D21995044
:1050100010BDC046B8060010034B0022190098339B
:1050200094310A601A607047B80600100122034BE1
:10503000943319684A401A607047C046B806001099
:10504000074B002219008C310A6001211A67054ABA
:1050500099501A009432126851424A41DA667047F8
:10506000B8060010AC07000070B5874B874DEC58B0
:10507000874BA210A41119570F231340581E0E2856
:105080003DD801F0B9FD0810171E223C283C3C2EEB
:105090003C3C3C323600002931DB002269184631A5
:1050A0000A70180070BD002929DB012369184631F8
:1050B0000B70F6E7002922DB0800FFF7CFFE012383
:1050C000EFE72000FFF796FFF9E7002917DB08005C
:1050D000FFF78EFDF3E7002911DB0800FFF780FDE5
:1050E000EDE72000FFF714FDE9E72000FFF7E8FCFB
:1050F000E5E7002903DB0800FFF760FFDFE7982AF8
:1051000000D19CE063DC382A00D186E03DDC1C2A1B
:1051100000D179E029DC162A70D021DC0123002A95
:10512000BFD0023B0C2ABCD1012398352B60B8E7D5
:10513000D63A1000222A15D801F05EFD901493147F
:1051400014149614141414141414141499149C1490
:1051500014149F14141414A2ACAF14B2B5B8BB004D
:10516000182A4ED001235B429BE72C2A52D007DC41
:10517000262A4CD0282AF5D100236B66013390E70C
:10518000362AEFD1FFF7D0FD99E7662A4ED00FDC23
:10519000562A48D007DC3C2A42D04C2AE2D1FFF7FD
:1051A000C5FE02237DE75C2ADCD1FFF791FB86E791
:1051B000762A41D006DC682A3BD06C2AD2D1FFF790
:1051C0009BFB7CE7882ACDD1FFF71EFC77E7F82A06
:1051D000C8DCD52AACDCBC2A3AD008DCA82A31D0FD
:1051E000B82A32D09C2ABDD1FFF726FC67E7C82A2F
:1051F00031D0CC2AB6D1FFF7D5FC60E7FFF722FD0E
:105200005DE7FFF71DFF5AE7FFF7E0FD57E7FFF700
:105210003FFD54E7FFF7E6FD51E701236B6640E7EA
:10522000FFF7ECFD4BE7FFF7F5FD48E7FFF7FEFD65
:1052300045E7FFF793FE42E7FFF704FE3FE7002351
:105240002B669BE701232B662BE7FFF7E5FE36E78E
:10525000FFF786FC33E7FFF7E9FE30E7FFF758FE7C
:105260002DE7FFF769FB2AE7FFF78CFE27E7FFF73B
:1052700041FE24E7FFF772FB21E7FFF791FE1EE7EF
:10528000FFF7F4FD1BE7C046C4070000B806001096
:1052900038AC0000FFF774FB11E7FFF783FB0EE764
:1052A000FFF7B2FC0BE7FFF70DFE08E7FFF7BAFCCC
:1052B00005E7FFF731FB02E770B51D4C1D4D1E4B96
:1052C0006259E25023008C331868FFF7E1F8E36E6F
:1052D0006051A3660023194DE36663510333184000
:1052E00002281FD0984220D0012818D0FFF7BCFE1A
:1052F00000280CDD6359002B04D122008C32136886
:105300001B1813602200903213681B181360FA22D6
:10531000D200A358002B01D0013BA35070BDFFF772
:1053200087FAE5E7FFF7EEF8E2E7FFF7AFFADFE726
:10533000B8060010C4070000CC070000AC0700004E
:105340000122034BDA66034A9A830F229A77704749
:10535000B80600100F0F000070B5F425074CED00E3
:1053600066592000064901F009FF6651FFF7E8FF82
:105370000123044A6366A35470BDC046B8060010FA
:10538000D40700009C0700007047000030B50D4DA9
:10539000049C28600C4801600C490A600C4A1360A8
:1053A0000C4B039A1A600C4B0C4A1C60F423DB0074
:1053B000D4500B4B0B4A1A600B4B0C4A13600C4A2F
:1053C000136030BD940E0010AC0E0010C80E00101B
:1053D000B40E0010D00E001024000010B80600100B
:1053E0008C0E001055550000895300009C0E0010D3
:1053F000CC0E0010014B18607047C046A80E00107C
:10540000084B10B51968084A002906D1074C2468D2
:105410002160106001221A6010BD11688842F8DA1C
:105420000800F6E7A00E0010A40E0010A80E001051
:10543000034B1B68002B01D1024A13607047C04622
:10544000980E0010A00E001070B51A4D2B00983366
:105450001B68002B0DD0184B1C6801231C40F52342
:10546000DB00EB58A34208D1144BEB58002B10D1B2
:1054700070BD2B0094331C68F1E7002C0BD1002B7E
:10548000F6D00F4B1B68002B0FD02100200098474F
:105490000BE0002CECD00A4B084E1B68002B02D00E
:1054A0002000A95998470023AB51F523DB00EC50AD
:1054B000DEE7C046B8060010900E0010A4070000FA
:1054C000940E0010054B10B51B68002B04D0044946
:1054D000044A01208958984710BDC046940E001018
:1054E000B8060010A40700000023F821054AC900EF
:1054F0001370054A53500549535004315350044A20
:1055000013707047B10E0010B8060010B407000009
:10551000B80E0010084B1860084B196000280AD01C
:1055200001230021064A1370064A1170064A0749F2
:105530008850074A13707047BC0E0010C00E001050
:10554000B10E0010B00E0010B4070000B806001035
:10555000B80E00102C4B73B51A682C4B11681868E4
:1055600081421AD000210091019112681A60284BE3
:105570001B688B4202D0684601A9984725490098CC
:105580000C68019A244BA04202D11C68944202D0BC
:105590000125224C257008601A60214C214BE358EC
:1055A000002B10D000231D49CB56002B0AD000221F
:1055B0001D4B9A56012A05D100220A701B490A7018
:1055C00002321A7073BD134B174D1868002807D0AC
:1055D0000023EB56002B03D10F4B1968FFF79AFFFE
:1055E0000023EB56114E022B08D10023104A3370D2
:1055F000A3502B700023F356E366E3E7002BF9D0AA
:105600000A20FFF7FDFEF5E7B40E00102C00001095
:10561000AC0E0010BC0E0010C00E0010B00E00103A
:10562000B8060010BC070000B80E0010B10E001044
:10563000B4070000F82370B5054CDB00E358002BDD
:1056400005D1E56E034AA350FFF784FFE56670BD00
:10565000B8060010BC070000084A094B11681B6817
:1056600010B5CB1A03D41360FFF7EEFE10BDFA237A
:105670005B001360034A13680133F4E7280000104D
:10568000D00E0010900E00100122034B1A60034B45
:10569000F432FF321A607047900E0010280000109C
:1056A00073B5040000250026134B00961B68019675
:1056B000B34218D101350220FAF73CFE0F4B1A68AD
:1056C0000F4B11681868814208D012681A60FFF702
:1056D000C3FF002C02D0013C002C02D0042DE2D1EB
:1056E0000124200076BD684601A99847009B002B45
:1056F000E0D03500DFE7C046AC0E0010B40E00105D
:10570000C40E0010F7B56C4B6C4C0500E050043330
:10571000E150230094331B680E00002B0ED1182893
:105720000AD1C32908D1664B1B680F2B04D116225E
:105730000E21644800F0F2F8FFF702FE00239D42BC
:1057400000D00A33F62231002800D200A350FFF720
:10575000E1FE5D4B5D4E1B6825001B688C35336098
:10576000FFF766FE012323671D3301930023009397
:10577000574B1B68002B14D0564F3B68002B10D0A2
:105780001B68002B56D03A681368013B1360524ADD
:105790001368002B05DD013B1360002B01D1FFF7DF
:1057A00047FEFFF789FD002807DA22002B689032B8
:1057B00001332B60136801331360484B009A484F44
:1057C0009A420CD040239A43464B9A4207D0464B0C
:1057D000009A9A4203D05333FF339A4211D1E359CE
:1057E000424A93420AD01A002020414982438A4209
:1057F00004D0402293433F4A934202D10A20FFF74C
:10580000FFFDE3593C4A00932B68934237D016DCE6
:1058100082221201934235D0384A934218D0019B1C
:10582000002B32DD013B0193236F002BA0D1FFF74A
:105830000BFEF7BD324B1B6898473B68A0E7314A27
:10584000934215D0304A9342E9D1FBF7F3FBE6E7E8
:10585000FBF702FCFFF736FEFAF716FE2B4B18603B
:10586000154BE0503368013B3360294B2B60D6E782
:10587000FAF764FDFFF708FFFFF724FECFE7FBF719
:10588000C5FFCCE7FBF758FBC9E7224B1B689847DD
:105890001E200D4B01901A681F4B11681868814239
:1058A000C2D012681A60FFF7C5FEFFF7D5FE144B91
:1058B0001B689847B8E7C046B4070000B806001058
:1058C00024000010F0060010B40E00102C00001090
:1058D000A00E0010A80E0010A40E00106E02000012
:1058E000C4070000260200007A020000FB0300004B
:1058F000CB030000A3030000490F00006A0C000066
:105900009C0E0010FA1300003A150000BC0E0010A7
:105910006F0C0000CC0E0010C40E0010F0B5012575
:10592000002A00DCF0BD03784C1E2B40002C01DA6D
:10593000013AF5E7065DDB0077083B43035533008A
:10594000013C2B40F2E730B59A4200DD30BD845C6B
:105950008D5C85548C540132F6E7F0B5060007A83B
:105960000578069801240078002A1DD0059CA342E2
:1059700004DD01231840069B1870F0BDD75CCC5C99
:10598000BC46644424180020A54201DC641B01309D
:10599000F4540133EAE7CA5C12180020954201DC96
:1059A0002000521BF2540133059A9342F3DDE0E7E5
:1059B000F7B50AAC2478089F0194099C2478002844
:1059C00039D00F25002933D0002A1ED1019E0F3275
:1059D000013E1640BB421ADCCA5C121B0024551C57
:1059E00001D132000134C2540133F3E7CD5C2E0003
:1059F000D55C751B2D1B0024A54204DA019C65199A
:105A00000F2425400E3CC5540133BB42EEDD01237B
:105A10001C40099B1C70F7BDD15C49420C1B002146
:105A20008C4203D00199091901242940C154013342
:105A3000BB42F1DDEBE7002919D0002A0ED1BB42B1
:105A4000E5DCCA5C0133141B013462425441F6E7C1
:105A5000C85CD55C0133401B041BE40FBB42F7DD7F
:105A6000D5E7D15C013349420C1B611E8C41BB421E
:105A7000F7DDCCE770B50125049C257000290BD11A
:105A80009A420BDC815C00290AD10132F8E7865C7E
:105A90008D5CAE4204D101329A42F8DD00232370BE
:105AA00070BD0B0030B5441C934207DB002423007B
:105AB000914200DC531A4018C45430BDE55CC55413
:105AC0000133F1E7130030B5441E8B4207DC00249C
:105AD00023008A4200DB8B1A8018C45430BDE55C79
:105AE000C554013BF1E70000F0B5114A01241378D9
:105AF000C15C53780B405A1E93410E499B010B60C9
:105B00000D4B00221F0001254A6012371A785E787B
:105B1000825C164202D04A682A434A6002336D0012
:105B2000BB42F3D1013404310B2CEAD10020F0BD8B
:105B30007201001068100010BE000010122230B573
:105B400005254A43324C01311319A25C5C78825C12
:105B50006943144204D05F242E4A52189470547042
:105B60009A78DC78825C144204D07C24294A52184A
:105B7000533214701A795C79825C144204D07C240C
:105B8000244A5218A33214709A79DC79825C144248
:105B900007D0204A5F2452181500A132A2352C707C
:105BA00014701A7A5C7A825C144204D07C24194AFC
:105BB0005218A03214709A7ADC7A825C144204D0B3
:105BC0007C24144A5218503214701A7B5C7B825C1D
:105BD000144207D00F4A5F24521815005132523533
:105BE0002C7014709A7BDC7B825C144204D02E24CF
:105BF000084A5218A43214701A7C5B7C825C1342EF
:105C000004D0044B59182723F4310B70002030BD09
:105C1000BE000010D80E0010F7B5040000262D4D70
:105C20002F00393F4F2220213800FDF7FDFF002EC5
:105C300002D07C233B702B7000210136A9755035B2
:105C4000052EEDD1244B2D2218003830027018009B
:105C500037300270A1209A705A70400032321A54C4
:105C60004220FF301A54053019541C4908784978ED
:105C7000205C014204D01900523353310A701A706B
:105C80000027390020000137FFF758FF0A2FF8D10D
:105C90000025134E0197134BAA00D1583378727820
:105CA000E35C114F1A420CD03800013501F090FA34
:105CB0000236092DEFD138000C4901F089FA052090
:105CC000FEBD0800FDF7E8FF019B0949181A0918F5
:105CD000EAE7C046110F0010D80E00107201001044
:105CE000AC000010540000101810001048AC000068
:105CF0009C000010014B18707047C046D70E001072
:105D00000020034B185642425041C0B218707047F1
:105D1000D60E0010014B40B218707047D50E00101F
:105D20000020014B18567047D50E001070B50C00BE
:105D3000C3050FD5CCB2D5B2A01DE91DC9B2C0B202
:105D4000FCF79AFB290005340831C9B2E0B2FCF730
:105D500093FB70BD0306FCD506320634D1B2022394
:105D60000122E0B2FCF79CFBF3E7012370B50600CB
:105D70000C001500184206D0D118E0180322C9B251
:105D8000C0B2FCF78DFB02231E4206D0E918201D8D
:105D90000122C9B2C0B2FCF783FB730707D5691DA6
:105DA000201D02230122C9B2C0B2FCF779FB3307E0
:105DB00007D5E91D601C01230322C9B2C0B2FCF75C
:105DC0006FFBF30606D5691D02230122C9B2E0B2BA
:105DD000FCF766FBB30606D5A91C02230122C9B253
:105DE000E0B2FCF75DFB730607D5291D01340123E2
:105DF0000322C9B2E0B2FCF753FB70BD064B07208B
:105E00001B785BB2002B06D1044B01381B785BB2C8
:105E1000002B00D118007047D50E0010D60E0010D0
:105E20001C4B10B51900DE314A8808881A49120443
:105E3000024300208A4222D1E3335A781C789978B1
:105E40001202DB7814430904144A21431B060B4356
:105E5000934214D1FFF7D2FF1149124C0978020086
:105E600049B22368104800290AD0023323600F2169
:105E70000E4BFCF797FB2368023B0120236010BD0B
:105E80000333236009210A4BFCF78CFB2368033B97
:105E9000F3E7C046B80600103D001D1111444C80C8
:105EA000D50E00101800001050AC0000DC8A000075
:105EB000EC8A0000F0B5A24B89B01C680394022C58
:105EC00003DD231F5A425A410392FFF797FF9D4B70
:105ED00006001B785BB25A1E93415B420293052C6D
:105EE0004CD0994B0193062C04D0984B0193984BBE
:105EF000042C47D00022974B05921B785BB293424B
:105F000005D007230393944B0193012305930023AA
:105F1000924C00930C3C00228E4B9A560823002A88
:105F200000D10433009A0127002A01D017005F43F3
:105F3000834B1B68022B11DD00227F2007AB5A70B8
:105F4000E36818404E281FDC212800D1CEE05DDC3C
:105F5000783213424ED01C2800D1CDE00123039AA1
:105F6000072A00D9DBE0100000F05AFE0D017F0186
:105F70000802D900D900D900D900000101235B42F1
:105F80000293774B0193B5E74F383028E6D800F0FD
:105F90003DFE6F00AD00E5FFE5FFE5FFB600E5FF64
:105FA000E5FFE5FFE5FFE5FFE5FF6C00B000E5FF7D
:105FB0009E00E5FFE5FFE5FFB300E5FFE5FFE5FF38
:105FC0007200E5FFE5FFE5FFE5FFE5FFE5FF750092
:105FD000E5FF8100E5FFA400E5FFAA00A700E5FFBB
:105FE000A7009500E5FFA100E5FFE5FF9800780018
:105FF000E5FF7E000728B1D800F008FE1400B0FFCE
:106000008400B0FFB0FFB0FF22004600232876D006
:1060100038380828A2D800F0E5FD2557A1A1A1A194
:10602000A14B4E00202207AB1A70019B32003900B1
:1060300007A8FCF7B7FA059B002B66D000238EE774
:10604000312207AB1A70009B022BEEDD7F236268C2
:106050001A40542A06D0009A032AE6DD226813402B
:10606000542BE2D14C2207ABDEE7322207ABDBE751
:10607000332207ABD8E7342207ABD5E7352207AB8D
:10608000D2E7362207ABCFE7372207ABCCE738227F
:1060900007ABC9E7392307AA1370009B062BC4DDA1
:1060A0007F23A1680B40232BBFD124331370BCE79F
:1060B000302207ABB8E72D2207ABB5E7412207AB8B
:1060C000B2E7422207ABAFE7432207ABACE744227B
:1060D00007ABA9E7452207ABA6E7462207ABA3E734
:1060E000482207ABA0E7502207AB9DE7522207AB3F
:1060F0009AE74F2207AB97E7552207AB94E74E226A
:1061000007AB91E7492207AB8EE7E368DA050FD5C5
:10611000029B14489A19019BF91DFCF743FA009B56
:106120000434013300930B2B00D0F4E609B0F0BD2A
:106130001B06F4D53200019B0B48F91DEDE7C04664
:10614000A8000010D60E0010C48A0000EC8A0000DF
:10615000E48A0000D50E0010DC8A000068100010F0
:10616000CC8A00005DAC000031750000002B04D02B
:1061700032003900E068FFF7F8FD32003900E068CE
:10618000FFF7D4FDCBE70123E2681A4205D0B81C23
:106190000522F1B2C0B2FCF783F9E3689B0707D58B
:1061A000711CF81D03230122C9B2C0B2FCF778F9B3
:1061B0000423E2681A4206D0711DF81D0122C9B2FB
:1061C000C0B2FCF76DF90822E368134208D0310031
:1061D000B81C09310123C9B2C0B2033AFCF760F917
:1061E000E368DB0607D5711D781C04230122C9B2C0
:1061F000C0B2FCF755F9E3689B0607D5711C781C03
:1062000003230122C9B2C0B2FCF74AF9E3685B0676
:1062100007D5311DB81C01230522C9B2C0B2FCF755
:106220003FF9E368DA0513D5029BFFB2F518EDB22A
:10623000290038000A310930C9B2C0B2FCF71CF994
:106240003B0009350A33E9B2D8B2FCF715F966E725
:106250001B0600D463E7310001230222093109370C
:10626000C9B2F8B2FCF71CF959E70122E3681342FE
:1062700012D0FDB2F1B20495A81C0D001300C0B2FB
:106280000432FCF70DF96B1CD9B2049B0322DD1C10
:10629000E8B20123FCF704F90222E368134206D0B6
:1062A000711CB81D0323C9B2C0B2FCF7F9F804236E
:1062B000E2681A4206D0711DB81D0222C9B2C0B2EE
:1062C000FCF7EEF80822E368134212D0FDB2F1B2F7
:1062D000A81C09310123C9B2C0B2033AFCF7E0F8A7
:1062E000F1B20831033501230322C9B2E8B2FCF749
:1062F000D7F8E368DB0607D5711D781C042302225A
:10630000C9B2C0B2FCF7CCF8E3689B0607D5711C94
:10631000781C03230222C9B2C0B2FCF7C1F8E368BB
:106320005B0612D5FDB2F3B2191DA81C012305228C
:10633000C9B2C0B2FCF7B4F8F3B20533D9B2032244
:1063400001230335E8B2FCF7ABF8E368DA055FD563
:10635000029BFFB2F518EDB2290038000223083184
:106360000A301A00C9B2C0B2FCF79AF83B000935EE
:106370000933E9B2D8B202231A0073E7E368DB07F6
:1063800006D5781C02230722F1B2C0B2FCF788F8C8
:106390000222E368134205D0B81D0623F1B2C0B251
:1063A000FCF77EF8E3685B0707D5311DB81D0623AF
:1063B0000222C9B2C0B2FCF773F80822E3681342A4
:1063C00007D0B118781C0223C9B2C0B2013AFCF759
:1063D00067F8E368DB0607D5311D781C0623022227
:1063E000C9B2C0B2FCF75CF8E3689B0606D5781C1E
:1063F00006230222F1B2C0B2FCF752F8E3685B0652
:10640000A3D5311D781C02230722C9B2C0B29AE776
:106410001B0600D483E6310009370831C9B2F8B24F
:10642000A9E7C046F7B52C4A2C4B12781B6852B22C
:106430002B4C0190002A27D0002B06D0012280216E
:10644000284B29485242FCF7ADF8012700257F422E
:10645000264BEB5C012B12DC019922788A5C617877
:1064600011420CD0224AA9008858224AA95C08226D
:106470008900002B00D13A001A4BFCF793F8013544
:106480000234092DE4D1F7BD1B4A0927127852B214
:10649000002A01D002277F42002B05D03A000021BC
:1064A000104B1148FCF77EF80025019A2378D35C45
:1064B00062781A420AD0114B1148E95CAB009C4645
:1064C00066463A00074B3058FCF76CF80135023449
:1064D000092DEAD1D7E7C046D50E00109004001070
:1064E000AC000010D48A0000DB740000B8AC0000DF
:1064F00030000010AFAC0000D60E0010C1AC0000A0
:106500007800001070B500F053FA00280CD0114B41
:1065100006241B7803265BB2002B09D0022332002D
:1065200000211800FBF7BCFF70BD01340F2CFBD01D
:106530003100200000F0EEFC2000CDB2310000F070
:1065400003FC2900C0B2FBF797FF092CEDD1023400
:10655000EEE7C046D50E001070B50D000400FFF741
:10656000C3FAFBF7E9FEFFF75BFC002806D1002D1C
:1065700001D0FFF79FFC2000FFF754FF094B1B7869
:10658000002B0ED02000FFF747FB002450252900E8
:106590006143054B0548C9180134FDF70EFB052C76
:1065A000F5D170BD75020010D80E00108179000081
:1065B00010B588B00400092101A8FDF779FF122069
:1065C0000A216844FDF774FF210001A8FFF7C4FF0A
:1065D00008B010BD10B5124B1B785BB2002B14D164
:1065E000002813D0FBF773FE0120FFF7E1FFFBF754
:1065F000DBFE00230B4AD356002B06DD013BDBB24A
:106600001370002B01D1FEF76FFF10BDFBF767FE83
:10661000054B1B78002BF8D00448FDF7CEFAF4E7C1
:10662000D70E0010D40E0010750200105FAC0000F1
:1066300010B5FBF797FE10BD70B50D0004000721E3
:10664000002D0BD0FDF728FB062156234143591A94
:10665000CB43DB171940012D00DD4910012220003A
:10666000024B5242FBF79EFF70BDC046DC8A000021
:10667000F0B589B0050000F0B7F98023002825D1D6
:10668000039300F0C7F943B201930C2B00D1CDE086
:106690002B78002B1CD0AB7804335BB20293012320
:1066A0005B420493002306AA5371019B0C2B13D168
:1066B0002B78092B13D12D2306AA13710122012156
:1066C0005E4B524207A8FBF76DFF08E05B00D7E77F
:1066D00001235B420293E4E7029B0C2BEBDC0127D6
:1066E0000C247F42049B0C3B1B19DBB20593019BDE
:1066F0000C2B0BD0AA78E31E9A4204DA029A63B2FA
:10670000934200D088E0042C00D885E0019AEB1C6D
:106710001B5D0C2A02D10F2B00D17DE0029861B2E3
:1067200007AA814202D12D2313700CE005292CD138
:1067300001990C2929D16978002926D02D21002B17
:1067400000D10D3911703E4BE6001B687642683669
:10675000022B52DC07AB1878203826284DD800F0E1
:106760004BFA484C4C4C4C4C4C4C4C4C4C4C4C3AD2
:106770004C4C384A1A2A2C2E303234364C4C4C4C65
:106780004C4C4C3C3E40424446003721092B00DC37
:1067900007395B18C8E75B203A003100FFF7E5FADC
:1067A000059B092B38D8180000F026FA3C36362E07
:1067B00036362E36362E4F20EEE76620ECE76D207B
:1067C000EAE77D20E8E70720E6E77F20E4E76F209F
:1067D000E2E73F20E0E74020DEE77720DCE77C20AF
:1067E000DAE73920D8E75E20D6E77920D4E77120B0
:1067F000D2E70020D0E70620CEE73A0031000F4B69
:1068000007A8FBF7CFFECBE7C0203A003100039B7F
:1068100040005840FFF78AFA013C022C00D061E7A3
:1068200009B0F0BD3A0031000398F3E71023EB56AE
:10683000049301235B42029334E7C046DC8A0000E4
:10684000A8000010002210B5094B9A56094B002AE7
:1068500004D007221100FBF7A5FE10BD0021064A57
:1068600051560622002900D1053A0C21F3E7C04613
:10687000D50E0010DC8A0000D60E001010B5040002
:10688000FBF75AFD0020FFF793FE2000FFF7DAFF29
:1068900010BD10B5FFF7D6FF10BD0000002370B586
:1068A000134A144C0D00A3500432A350083AA350CD
:1068B00022008C3210600122E3662267236F002BD6
:1068C00004D026008C363368AB4203D1FEF7B8FB08
:1068D000002070BDFEF7F0FC0028EFDA22003368DC
:1068E000903201333360136801331360E6E7C0462A
:1068F000B4070000B8060010F0B50026274CA3B07E
:106900000090019115002100782204A8FDF76BF991
:10691000234F0722390002A8FDF765F90E220099DE
:1069200020482666FDF75FF9019B0E223B7031007F
:106930001D48FDF779F931001C48A667FFF7AEFF47
:106940002300CC331A780F239A432300C02A1ED188
:1069500045331B782B700023C02A04D123004E330B
:106960001B785A1E93416B70636D2100AB700E2231
:10697000E81CFDF738F904A978222000FDF733F967
:106980000722380002A9FDF72EF923B0F0BD4933E4
:106990001B78591E8B41DBB2DCE7C046B8060010FD
:1069A00085070010F0060010FE0600109A11000086
:1069B000034B04489B6D1841012318407047C046A3
:1069C000B8060010F70200000200103A0300B82ACF
:1069D00005D80448C0181038007840B2704701202C
:1069E0004042FBE774010010C920024B1856C00F4B
:1069F0007047C046B8060010014B46331878704700
:106A0000B8060010024B986D033843425841704756
:106A1000B8060010024BCC33187800097047C04606
:106A2000B8060010024BCC3318780F23184070477B
:106A3000B8060010074B0F20CB331A781300120949
:106A40000340801A80000422082B01D805339A10D5
:106A500080187047B8060010024BCA3318788006B9
:106A6000400F7047B806001003000020052B05D822
:106A7000034AC93210781841012318407047C046B4
:106A8000B806001010B5FFF793FF002815D00C4A88
:106A90001300B8331B78926D1B09012B07D10A2014
:106AA000072A09D01800042A06D10C2004E0022B82
:106AB000F8D10B20062AF5D110BD01204042FBE79A
:106AC000B80600100B4B30B51A00B93215780F24F8
:106AD000290000222140254202D02F3101700132CD
:106AE000B8331B781B0902D02F33835401320023A3
:106AF000835430BDB8060010034B1B18C03B1B78F5
:106B00000248C0187047C04634B1000043B10000CD
:106B100070B504000D002878002801D1207070BDE8
:106B2000BF2803D8207001340135F4E7FFF7E4FFF4
:106B3000060001002000FDF7B7F83000FDF7ACF8C3
:106B40002418F1E70268030010B50B488A4212DCF2
:106B50005C688C420FDB3F20891A8A11014098182B
:106B6000047C05488C4206DD9868DB6892009B58DF
:106B700080585B5CC01810BD878B000010B5010009
:106B80000148FFF7DFFF10BD20B1000010B5040081
:106B90000800FFF7F3FF01002000FFF7B9FF10BD69
:106BA000FEE7FEE710B50A4A0A4B0B498B4207D3B2
:106BB00000210A4B0A4A934207D3FAF7D1FFFEE7B6
:106BC0001078013218700133F0E719700133F2E7E1
:106BD0009CB10000000000102D02001030020010D7
:106BE0009410001002B47146490849000956490042
:106BF0008E4402BC7047C04602B471464908490041
:106C0000095C49008E4402BC7047C04603B471461B
:106C1000490840004900095E49008E4403BC7047A2
:106C200003B47146490840004900095A49008E449E
:106C300003BC7047002243088B4274D303098B4284
:106C40005FD3030A8B4244D3030B8B4228D3030C3C
:106C50008B420DD3FF22090212BA030C8B4202D3DE
:106C60001212090265D0030B8B4219D300E0090A06
:106C7000C30B8B4201D3CB03C01A5241830B8B420F
:106C800001D38B03C01A5241430B8B4201D34B03F8
:106C9000C01A5241030B8B4201D30B03C01A52415D
:106CA000C30A8B4201D3CB02C01A5241830A8B42E2
:106CB00001D38B02C01A5241430A8B4201D34B02CB
:106CC000C01A5241030A8B4201D30B02C01A52412F
:106CD000CDD2C3098B4201D3CB01C01A52418309E3
:106CE0008B4201D38B01C01A524143098B4201D31D
:106CF0004B01C01A524103098B4201D30B01C01A48
:106D00005241C3088B4201D3CB00C01A52418308C1
:106D10008B4201D38B00C01A524143088B4201D3EE
:106D20004B00C01A5241411A00D20146524110464E
:106D30007047FFE701B5002000F0F0F802BDC04643
:106D40000029F7D076E7704703460B437FD4002233
:106D500043088B4274D303098B425FD3030A8B42EF
:106D600044D3030B8B4228D3030C8B420DD3FF2259
:106D7000090212BA030C8B4202D31212090265D027
:106D8000030B8B4219D300E0090AC30B8B4201D3DA
:106D9000CB03C01A5241830B8B4201D38B03C01A21
:106DA0005241430B8B4201D34B03C01A5241030B98
:106DB0008B4201D30B03C01A5241C30A8B4201D349
:106DC000CB02C01A5241830A8B4201D38B02C01AF4
:106DD0005241430A8B4201D34B02C01A5241030A6B
:106DE0008B4201D30B02C01A5241CDD2C3098B4250
:106DF00001D3CB01C01A524183098B4201D38B01CD
:106E0000C01A524143098B4201D34B01C01A52416F
:106E100003098B4201D30B01C01A5241C3088B42B4
:106E200001D3CB00C01A524183088B4201D38B009F
:106E3000C01A524143088B4201D34B00C01A524141
:106E4000411A00D201465241104670475DE0CA0F18
:106E500000D04942031000D34042534000229C46D8
:106E600003098B422DD3030A8B4212D3FC228901E2
:106E700012BA030A8B420CD3890192118B4208D3B8
:106E8000890192118B4204D389013AD0921100E01A
:106E90008909C3098B4201D3CB01C01A524183092E
:106EA0008B4201D38B01C01A524143098B4201D35B
:106EB0004B01C01A524103098B4201D30B01C01A86
:106EC0005241C3088B4201D3CB00C01A5241830800
:106ED0008B4201D38B00C01A5241D9D243088B4256
:106EE00001D34B00C01A5241411A00D201466346F9
:106EF00052415B10104601D34042002B00D549425D
:106F0000704763465B1000D3404201B5002000F09B
:106F100005F802BD0029F8D016E770477047C04653
:106F2000D0400B00D1409C46203AD34018435242F7
:106F300063469340184370479140030090409C463D
:106F4000203A9340194352426346D3401943704755
:106F5000002B11D1002A0FD1002900D1002802D026
:106F60000021C943080007B4024802A1401802905A
:106F700003BDC046A9FFFFFF03B4684601B50298F0
:106F800000F006F8019B9E4602B00CBC7047C0465C
:106F9000F0B557464E464546DE46E0B504000D00C6
:106FA0009246994683B08B4230D82DD04946504600
:106FB00000F0BAF829000600200000F0B5F8331AF6
:106FC0009846203B9B4633D45A465346934042460C
:106FD0001F00534693401E00AF423AD8AF4200D143
:106FE00078E05B46A41BBD41002B00DA75E000226F
:106FF00000230092019301235A46934001930123F9
:1070000042469340009328E08242CFD900220023D9
:10701000009201930C9B002B01D01C605D600098D6
:10702000019903B0F0BCBB46B246A946A046F0BDEC
:10703000424620239B1A5246DA40414613004A46F4
:107040008A40170042461F43534693401E00AF42FA
:10705000C4D900220023009201934346002BD9D0CB
:10706000FB0772081A4346467B080EE0AB4201D18B
:10707000A2420CD8A41A9D41012024196D4100217F
:10708000013E24184D41002E06D0AB42EED9013E00
:1070900024196D41002EF8D1009801995B46001922
:1070A0006941002B24DB2B005A464446D3402A007A
:1070B000E2401C005B461500002B2ADB26009E40A8
:1070C000330026004746BE403200801A99410090A6
:1070D00001919FE7A342BCD883E7424620230021C9
:1070E0009B1A0022009101920122DA40019286E768
:1070F000424620239B1A2A0046469A402300F3402A
:10710000444613432A00E2401C005B461500002B56
:10711000D4DA42462F002023260097409B1ADE40F7
:107120003B003343CDE7C04610B5002903D100F042
:1071300007F8203002E0080000F002F810BDC04659
:107140001C2101231B04984201D3000C10391B0A97
:10715000984201D3000A08391B09984201D300095B
:10716000043902A2105C40187047C04604030202B2
:1071700001010101000000000000000010B50A003C
:107180000021FCF751FD10BD30B5032A0CD90300D6
:107190000B439B0719D103680C68A34215D1043A2D
:1071A00004300431032AF6D8551E002A0BD00023E0
:1071B00003E05A1C9D4206D01300C25CCC5CA24284
:1071C000F7D0101B00E0002030BD551EEFE7C04691
:1071D00070B50400830716D102680E4B0E4DD3180C
:1071E00093432B420FD142680A4B0430D318934388
:1071F0002B4208D14268074B0430D31893432B42EB
:10720000F1D000E001300378002BFBD1FCF74CFDFE
:10721000200070BDFFFEFEFE808080805B40253038
:107220003278253032785D0D0A00444D3136002524
:10723000732025730D0A0053455249414C20434F9A
:107240004E534F4C45007265616479000D0A4279D6
:10725000652E2E2E0D0A004E4F00203F005633346F
:10726000002573202573202025694D485A002020D1
:1072700025692E253033695600202573525443204A
:1072800000524553455420544F2041424F52540020
:10729000524541445920464F5220464C415348499B
:1072A0004E47004C43443A25303269202D20256951
:1072B00000505245535320454E54455220544F20C0
:1072C000534156450053574953534D4943524F5329
:1072D0002028432920323031302D323032350025FC
:1072E000633120484F5552002D00525443205245DF
:1072F0004144204641494C005F005052474D2054C4
:107300004F50007E004E554C4C00537461727420F7
:10731000626F6F746C6F616465723F00454E5445D7
:1073200052206966204F4B20656C73652061626F47
:1073300072740053657475703A00507265737320EF
:1073400061206B6579004C656176696E67207365B5
:10735000747570206D656E750089004B6579202508
:107360007800556E75736564206B65790030313235
:107370003334353637383941424344454600534863
:107380004F57204845580053484F57204445430025
:1073900053484F57204F43540053484F57204249BA
:1073A0004E005B40313830305D0D0A005B403030BC
:1073B00030305D0D0A007475726E6564206F6E006A
:1073C0003C52455345543E0D0A00410044697370D8
:1073D0006C617920646174652F74696D6500426524
:1073E0006E63686D61726B0053657269616C2063D6
:1073F0006F6E736F6C6500537461727420626F6F8F
:10740000746C6F616465720053797374656D206983
:107410006E666F004C434420636F6E7472617374C8
:10742000004C434420636F6E747261737420726504
:107430007365740053544F00525443202D3120681B
:107440006F75720052434C00525443202B31206818
:107450006F7572003100312D6C696E65206469733F
:10746000706C6179003200322D6C696E6520646940
:1074700073706C61790037004379636C6520666FC7
:107480006E74003900546F67676C65204350552057
:10749000737065656400C3B7004B6579626F617294
:1074A0006420746573740053656C6620746573742E
:1074B00000506F776572207265736574002B00450C
:1074C0006E646C657373207465737400546F6767C2
:1074D0006C6520646F742F636F6D6D61004753425C
:1074E0000041646A75737420646174652F74696DFA
:1074F000650047544F00546F67676C6520616E6E7E
:10750000756E636961746F7220706F73004C424CCA
:1075100020005346200043462000463F20004754A9
:107520004F2000475342200052434C200052434C0E
:10753000202E0053544F200053544F202E00574903
:107540004E444F572000464C4F41542000330038E2
:107550000028692900434C454152205052474D00B4
:10756000496E76616C6964206D6174682F44697638
:10757000206279203000466C61672F57696E646F16
:10758000772F466C6F61742F47544F2E00496D70F2
:10759000726F70657220426974204E756D626572FB
:1075A00000496D70726F70657220526567204E756C
:1075B0006D62657200426164204C696E6520232F04
:1075C0004C6162656C2063616C6C00537562722063
:1075D0006C6576656C20746F6F206465657000491A
:1075E0006E76616C69642052656720436F6E7465C6
:1075F0006E74730060750000767500008D75000074
:10760000A1750000B5750000CB750000DF750000A6
:10761000FA00FB00FC00FD00FE00FF00F700F80090
:10762000F900CF00F9FFFAFFC100C200C300C40097
:10763000F400F500F600CE00FFFFFFFFC500CA0012
:10764000FFFFC600F100F200F300CD00FFFFFFFFD7
:10765000FFFFF6FFF8FFFFFFF000C900CB00CC00F2
:10766000EA00EB00EC00ED00EE00EF00E700E800C0
:10767000E900BF00B900E000FFFFFFFFFFFFFFFFD1
:10768000E400E500E600BE00DCFFDDFFD8FFBA0045
:10769000FFFFF4FFE100E200E300BD00FFFFFFFF9A
:1076A000FFFFB800F3FFFFFFFFFFFFFFBB00BC00C1
:1076B000DA00DB00DC00DD00DE00DF00D700D800F0
:1076C000D900AF00D400FEFFA100A200A300A400D7
:1076D000FDFFFCFFFBFFAE00FFFFFFFFA500AA00C0
:1076E000C000A600D100D200D300AD00FFFFFFFF15
:1076F000FFFFA800A700FFFFD000A900AB00AC006F
:10770000E4FFE3FFE2FFE1FFE0FFDFFFE7FFE6FF6B
:10771000E5FFFFFFFFFFFFFFC100C200C300C40081
:10772000EAFFE9FFE8FFFFFFDCFFDDFFFFFFFFFFF0
:10773000FFFFFFFFEDFFECFFEBFFFFFFFFFFFFFF92
:10774000FFFFFFFFFFFFFFFFEEFFDEFFFFFFFFFF7B
:107750000000031C10C001071C10FF01071C10FFD4
:1077600001371C10C001071C300000300000FF0171
:10777000071C3000000000010001000100000000B3
:1077800003000000030304030403010201000000DE
:107790000D75000012750000167500001A750000C6
:1077A0001E75000023750000287500002D7500006F
:1077B00033750000387500003E7500004675000006
:1077C00088750000878B0000878B0000878B000086
:1077D0007475000054740000657400004D7500005D
:1077E0005F720000DD7200002D72000076740000F0
:1077F0004F75000083740000CA730000DF7400003E
:107800008E73000079AC0000447200007C730000AD
:10781000317500000D8E000051750000878B00004F
:10782000878B0000878B000055750000878B000058
:10783000878B0000878B000011000000CA730000D6
:10784000CC73000012000000DF740000DE73000043
:10785000130000008E730000E873000014000000A5
:1078600079AC0000F77300001500000044720000BE
:1078700008740000160000007C73000014740000FF
:10788000260000009E7300002174000044000000E8
:107890003474000038740000450000004474000097
:1078A0004874000037000000547400005674000053
:1078B00038000000657400006774000017000000C5
:1078C00076740000787400001900000083740000D2
:1078D0008574000010000000967400009974000088
:1078E0002000000060730000A7740000300000005A
:1078F000E8720000B174000040000000BD74000098
:10790000BF7400004800000031750000CC74000016
:1079100021000000DD740000E1740000220000007E
:10792000F2740000F6740000FF000000878B000076
:10793000878B0000426164206E756D6265722E0D4A
:107940000A004241543A2025696D560D0A000D0A7D
:107950002530327820200057616974696E6720668F
:107960006F7220646174612E2E2E0D0A00426164D4
:10797000206D6F64656C0D0A004F4B0052656164A9
:107980002025730D0A004641494C4544006F666648
:10799000004C43442064656275672025730D0A001E
:1079A0004B4244206F75747075742025730D0A0066
:1079B000436F6E736F6C652074696D656F757420AD
:1079C00073657420746F202569206D696E75746508
:1079D000730D0A0074776F006F6E65005361792034
:1079E000626F6F746C6F61646572202573206D6FB8
:1079F00072652074696D652573202E2E2E0D0A0088
:107A00004C61756E6368696E6720626F6F746C6F2E
:107A100061646572202E2E2E0D0A00000000005CAD
:107A2000000C000C7C287C7C447C241048285408E2
:107A3000000C003844004438002010081038108032
:107A40004000101010004000201008384438007C1E
:107A5000006454484454281C107C4C54243854204E
:107A600004740C285428085438005000805000102A
:107A70002844282828442810045408384C5C7814DA
:107A8000787C54283844447C44387C54447C140426
:107A90003844347C107C007C0020403C7C106C7CA2
:107AA00040407C087C7C047C7C447C7C140838440A
:107AB000787C1468485424047C047C407C3C403C22
:107AC0007C207C6C106C1C601C64544C7C44000852
:107AD0001020447C0008040880808004080078445A
:107AE00078784478784478784478784478781414AE
:107AF00048543C000503050000BE0405000E000EBE
:107B0000050528FE28FE2805054854FE54240505D1
:107B1000462610C8C405056C92AA44A00305000AB5
:107B2000060405003844820405008244380505280F
:107B3000107C1028050510107C1010030500A060B3
:107B400005051010101010030500C0C00505804089
:107B500020100805057CA2928A7C04050084FE8022
:107B60000505C4A292928C0505449292926C05057B
:107B7000302824FE2005054E8A8A8A7205057894ED
:107B8000929260050502E2120A0605056C92929235
:107B90006C05050C9292523C0305006C6C030500C9
:107BA000AC6C0405102844820505282828282804E0
:107BB000058244281005050402A2120C05056492F2
:107BC000F2827C0505FC121212FC0505FE929292CF
:107BD0006C05057C828282440505FE82824438055C
:107BE00005FE929292820505FE1212120205057C94
:107BF0008282A2E40505FE101010FE04050082FE3C
:107C0000820505608080807E0505FE10284482057F
:107C100005FE808080800505FE041804FE0505FE33
:107C2000081020FE05057C8282827C0505FE12126A
:107C3000120C05057C82A242BC0505FE1232528C54
:107C400005054C9292926405050202FE02020505AA
:107C50007E8080807E05050E30C0300E0505FE401A
:107C60003040FE0505C6281028C605050608F008A0
:107C7000060505C2A2928A86040500FE82820505D9
:107C800008102040800405008282FE0505080402D9
:107C90000408050580808080800405000204080532
:107CA0000540A8A8A8F00505FE9090906004057016
:107CB000888888050560909090FE050570A8A8A8A2
:107CC0003005058888FC8A8A050510A8A8A87805CB
:107CD00005FE101010E005058888FA808004050074
:107CE000888A780505FE20205088050502027E80DE
:107CF000800505F8083008F00505F8080808F005C3
:107D00000570888888700505F82828281005051052
:107D1000282828F80505F810080808050590A8A8DF
:107D2000A848050508087E8888050578808040F801
:107D300005051860806018050538C030C038050595
:107D40008850205088050518A0A0A078050588C88F
:107D5000A89888040500106C8203050000FE040545
:107D600000826C10050520101020100005050590FC
:107D70005060A090050590A0402010050594546423
:107D8000A494050594A44424140505905462A49079
:107D9000050590A44224100505A0B0A8A4A20505DD
:107DA000A2A4A8B0A005052868382C28050510381D
:107DB0005410100505101054381005050804FE0471
:107DC0000805052040FE402003050030300505442D
:107DD0002810284405051010541010040500243EF6
:107DE000200305322A240505120A0C141205050881
:107DF0000808003E05052040FE0202050540807C83
:107E0000020403052AC42A050582C6AA92C60505EE
:107E1000887808F8880505609090701005057C92B8
:107E200092927C050580C0A090F804050C12120CFB
:107E300004050088FA8004057C545444050580003C
:107E40008000800305222A14040518143E10000542
:107E50000000040603000000007F01070400000783
:107E6000000000070B064400FF0144004400FF012E
:107E70004409058C009200FF019200620C06860006
:107E8000460020001000880184010C06EE0011015C
:107E900011012E01C0006001050300000000070968
:107EA0000500000000010182007C080400007C0045
:107EB0008200010109051000540038005400100927
:107EC00005100010007C0010001006030000800563
:107ED00080030B06100010001000100010001006A8
:107EE0000300008001800109050000C00030000C83
:107EF00000030B06FE000101010101010101FE0C5E
:107F000006000004010201FF01000100010C0682CD
:107F10000141012101210111010E010B0682000125
:107F200001110111011101EE0B063000280024009F
:107F30002200FF01200B068F000901090109010938
:107F400001F10B06FC001201110111011101E00BFE
:107F50000601000100E10111000900070B06EE0017
:107F60001101110111011101EE0B060E0011011199
:107F700001110191007E060300009801980106039B
:107F80000000980598030A051000280044008200AC
:107F900001010B06280028002800280028002809D5
:107FA00005010182004400280010090502000100BB
:107FB000610111000E0B06FE0001011901250129C6
:107FC00001BE0C06FE011100110011001100FE019E
:107FD0000B06FF011101110111011101EE0B06FE4B
:107FE000000101010101010101820B06FF010101F4
:107FF000010101010101FE0C06FF01110111011136
:1080000001110101010B06FF011100110011001106
:1080100000010B06FE000101010111011101F20C2A
:1080200006FF011000100010001000FF010A0501FA
:10803000010101FF01010101010B068000000100A7
:108040000100010001FF0C06FF01100028004400A0
:10805000820001010C06FF01000100010001000186
:1080600000010C06FF010400180018000400FF01C5
:108070000C06FF010400080010002000FF010B06A1
:10808000FE000101010101010101FE0B06FF0111CA
:10809000001100110011000E0C06FE00010101018B
:1080A000410181007E010C06FF01110031005100E9
:1080B00091000E010B068E00110111011101110139
:1080C000E2090501000100FF010100010B06FF00AC
:1080D0000001000100010001FF0B061F006000808D
:1080E00001800160001F0C06FF01400030003000DD
:1080F0004000FF010C06C3012400180018002400F2
:10810000C301090507000800F0010800070C06C1BB
:108110000121011101090105010301000406030009
:108120000000007F010704000007000000070B06A5
:108130004400FF0144004400FF014409058C009203
:1081400000FF019200620C0686004600200010002D
:10815000880184010C06EE00110111012E01C000FE
:108160006001050300000000070905000000000190
:108170000182007C080400007C00820001010905E6
:108180001000540038005400100905100010007C45
:108190000010001006030000800580030B0610008D
:1081A0001000100010001000100603000080018075
:1081B0000109050000C00030000C00030B06FE00A2
:1081C0002101110109010501FE0C06000004010254
:1081D00001FF01000100010C068201410121012182
:1081E0000111010E010B06820001011101110111A3
:1081F00001EE0B063000280024002200FF01200BB6
:10820000068F000901090109010901F10B06FC00B3
:108210001201110111011101E00B0601000100E141
:108220000111000900070B06EE00110111011101F7
:108230001101EE0B060E0011011101110191007EDA
:1082400006030000980198010603000098059803B2
:108250000A05100028004400820001010B062800D6
:108260002800280028002800280905010182004470
:1082700000280010090502000100610111000E0B29
:1082800006FE000101190125012901BE0C06FE01AF
:108290001100110011001100FE010B06FF01110178
:1082A000110111011101EE0B06FE00010101010196
:1082B000010101820B06FF01010101010101010120
:1082C000FE0C06FF01110111011101110101010B49
:1082D00006FF011100110011001100010B06FE0044
:1082E0000101010111011101F20C06FF0110001042
:1082F0000010001000FF010A0501010101FF01014A
:108300000101010B0680000001000100010001FFD6
:108310000C06FF01100028004400820001010C0639
:10832000FF01000100010001000100010C06FF0136
:108330000400180018000400FF010C06FF010400EF
:10834000080010002000FF010B06FE0001010101E2
:1083500001010101FE0B06FF0111001100110011C6
:10836000000E0C06FE0001010101410181007E01A9
:108370000C06FF0111003100510091000E010B06A7
:108380008E001101110111011101E2090501000125
:1083900000FF010100010B06FF00000100010001C8
:1083A0000001FF0B061F0060008001800160001FBC
:1083B0000C06FF014000300030004000FF010C06B9
:1083C000C3012400180018002400C3010905070098
:1083D0000800F0010800070C06C101210111010984
:1083E00001050103010007080400000000BF01BFF0
:1083F000010905000007000700070007130A000035
:108400002000E400FC003F00E700FC003F002700E4
:10841000040F0800000C011E01FF03FF032201E20C
:1084200001C2190D00000E001F0011019101FF0093
:108430007E00FC00FE0113011101F001E0140A00AE
:1084400000EE00FF0111011101BF01EE00E001305B
:10845000011001050300000F000F0A050000F800DD
:10846000FE03070701040B060000000001040707D4
:10847000FE03F80F08000000000A000E001F001F96
:10848000000E000A11090000100010001000FE008C
:10849000FE00100010001008040000000480078097
:1084A000030D070000100010001000100010001055
:1084B000080400000000800180010D07000C000F7F
:1084C000C003F0003C000F00030F080000FE00FF97
:1084D00001010101010101FF01FE1008000000007F
:1084E00002010201FF01FF0100010001100800006C
:1084F0008601C7016101210131011F010E010F0831
:10850000000082008301110111011101FF01EE1130
:10851000090000300038002C002600FF01FF012078
:1085200000200F08000080009F011F0111011101B0
:10853000F101E10F080000FC00FE010B0109010937
:1085400001F901F00F08000001000100C101F10173
:108550003D000F00030F080000EE00FF01110111A4
:10856000011101FF01EE0F0800001E003F01210173
:108570002101A101FF007E0804000000008C018C95
:10858000010804000000048C078C0312090000207D
:108590000070005000D80088008C01040104011113
:1085A00009000048004800480048004800480048CA
:1085B000004811090000040104018C018800D80062
:1085C00050007000200D07000002000300B101B947
:1085D000010F0006190D0000F800FC010603FB0660
:1085E000FD0505050505FD05FF050601FC01F81261
:1085F0000900008001F0017C004F004F007C00F07A
:108600000180010F080000FF01FF01110111011F8E
:1086100001FE01E0110900007C00FE008301010160
:108620000101010183018211090000FF01FF010125
:1086300001010101018301FE007C10080000FF011F
:10864000FF01110111011101110111010F080000B9
:10865000FF01FF01110011001100110001120900BA
:10866000007C00FE008301010121012101E301E200
:108670000112090000FF01FF01100010001000109E
:1086800000FF01FF010A0500000101FF01FF0101D8
:10869000010B060001000101010101FF01FF1008AB
:1086A0000000FF01FF0138006C00C60083010101DA
:1086B00010080000FF01FF0100010001000100019E
:1086C0000001160B0000FF01FF010F003C00F0004D
:1086D000F0003C000F00FF01FF0112090000FF0144
:1086E000FF010F001C007000E001FF01FF01130AF1
:1086F00000007C00FE0083010101010101018301F2
:10870000FE007C0F080000FF01FF01210021002175
:10871000003F001E140A00007C00FE0083010101DE
:10872000010101038307FE047C0412090000FF011C
:10873000FF01210021007100DF008E0100011109FD
:1087400000008E009F011101110111011101F301BF
:10875000E211090000010001000100FF01FF010119
:1087600000010001110900007F00FF0080010001ED
:1087700000018001FF007F1109000007001F007841
:1087800000E001E00178001F0007190D00000F0054
:108790007F00F001E0017C001F001F007C00E00171
:1087A000F0017F000F120900008301C7016C00383F
:1087B0000038006C00C701830111090000010007A7
:1087C000001E00F801F8011E000700011209000058
:1087D0008101C1016101310119010D01070103018D
:1087E0000004040200007F010905000007000000EA
:1087F0000000070B064400FF0144004400FF014451
:108800000B0600008C001201FF032201C40D078239
:108810000045002500920048014401820C0600003A
:10882000E60019012601C000200107040000000035
:10883000010002080400000000FE0101020804001B
:108840000000000102FE010B06000088005000201D
:10885000005000880B06000020002000F8002000D7
:108860002006030000000400020B06000020002088
:108870000020002000200603000000000001090580
:108880000000800160001800060B060000FE0001D9
:108890000101010101FE0804000002000200FF01C5
:1088A0000C06000082014101210111010E010B069D
:1088B00000008200010111011101EE0B06000060B1
:1088C0000058004600FF01400B0600009F00090110
:1088D00009010901F10B060000FE0011011101114F
:1088E00001E20B0600000100C10131000D00030B85
:1088F000060000EE00110111011101EE0B0600004F
:108900008E00110111011101FE0804000000008C0D
:10891000018C01080400000000000208010A0500A3
:108920000020005000880004010B06000050005099
:10893000005000500050090500000401880050005C
:10894000200B06000002000100610111000E0D075E
:108950007800860132014902390242027C0E07800A
:108960000170004C0043004C00700080010B0600B9
:1089700000FF01110111011101EE0B06FE000101C2
:10898000010101010101820B06FF01010101010149
:108990000182007C0C060000FF0111011101110190
:1089A00001010B060000FF01110011001100010C74
:1089B00006FE000101010111019100F2010C06FF08
:1089C000011000100010001000FF0108040000005A
:1089D000000000FF010704C00000010001FF0E07B6
:1089E0000000FF01180024004200810000010C0675
:1089F0000000FF0100010001000100010E07FF015E
:108A00000C003000C00030000C00FF010C06FF011C
:108A1000060018002000C000FF010B06FE00010147
:108A2000010101010101FE0B06FF011100110011FE
:108A30000011000E0C06FE0001010101410181013F
:108A4000FE020C06FF011100110011002900C601F1
:108A50000B0600008E00110111011101E20B06004E
:108A60000001000100FF010100010B06FF000001F1
:108A7000000100010001FF0D0703001C00600080E1
:108A80000160001C00030D071F00600080017C00D6
:108A9000800160001F0E0783014400280010002899
:108AA00000440083010D07030004000800F00108E2
:108AB000000400030E078101410121011101090198
:108AC000050103010D0C205AE58300000D0C205A0E
:108AD000E0870000030720671B7A0000050820A23A
:108AE000F37A0000060B205A1B810000060B205A67
:108AF000517E00002024282C383C4044484C18115A
:108B000010133831303378717073C8C1C0C3888195
:108B1000808384848782C5C4C7C2757477723534F4
:108B200037321514171200070008000A0100020767
:108B300002080201000301090304020402050305FF
:108B400000064669726D776172652025735F563342
:108B5000340D0A00252D3130732025732573000D47
:108B60000A5479706520273C636F6D6D616E643EB9
:108B7000203F2720666F7220706172616D730D0A4D
:108B80000025730D0A0D0A00564F594147455220E2
:108B90003E3E200025630048656C70004E6F2070DB
:108BA0006172616D73004B6579207072657373003B
:108BB0003C6B6579313E203C6B6579323E202E2E30
:108BC0002E0044756D70206D656D6F7279004C6F6D
:108BD0006164206D656D6F727900637400436F6E20
:108BE000736F6C652074696D656F7574003C6D6999
:108BF0006E757465733E00496E766F6B6520426FCB
:108C00006F746C6F6164657200536179207468726F
:108C100065652074696D6573004765742074696DBE
:108C200065005365742074696D65003C5959595944
:108C30004D4D44443E203C48484D4D53533E0074F6
:108C400064005570646174652074696D65003C6FE3
:108C500066667365745F696E5F6D696E7574657362
:108C60003E006B6200546F67676C65206B657962CC
:108C70006F617264206F757470757420746F2063F7
:108C80006F6E736F6C6500546F67676C6520646905
:108C900073706C6179206F757470757420746F20B7
:108CA000636F6E736F6C65005265616420626174FE
:108CB0007465727920766F6C7461676500000000DE
:108CC0005B72000000000000092D0000978B00007F
:108CD0009C8B0000DD750000FF0000006520000097
:108CE000A68B0000B08B0000F98D00000000000092
:108CF0008D1E0000C28B00009C8B0000D88D0000F0
:108D000000000000311F0000CE8B00009C8B000093
:108D1000DA8B00000100000015210000DD8B00004F
:108D2000ED8B0000FD7300000000000051210000E9
:108D3000F78B0000098C0000DB8B000000000000B6
:108D4000B11D0000198C00009C8B0000F175000023
:108D500002000000111E0000228C00002B8C00007D
:108D60003F8C0000010000004D1E0000428C0000FE
:108D70004E8C0000628C000000000000E920000022
:108D8000658C00009C8B00009474000000000000C3
:108D9000BD200000878C00009C8B0000638C0000CD
:108DA000000000009D1D0000A88C00009C8B0000AE
:108DB0000D0A413A2000202025633A20000D0A5375
:108DC0003A20000D0A4D3A20002020473A20253055
:108DD00032780D0A006661696C00253034692D25F2
:108DE0003032692D2530326920253032693A2530FC
:108DF00032693A25303269202573004D4F4E0054B8
:108E000055450057454400544855004652490053C3
:108E100041540053554E0000FB8D0000FF8D0000B3
:108E2000038E0000078E00000B8E00000F8E0000E6
:108E3000138E0000878B0000CF95135AB6566466D8
:108E40001595EEFE1EDE2FDF18213F871AD8B88257
:108E5000D02C611FB688ABBF3B01502419C462E31C
:108E6000BFCF0C20DA10DB1E3BE7E33451BF976B1A
:108E70009B01A3670C809D130A13EDEFB4893DB4E9
:108E80008E99AF2382EFE5A54E00C0000077ECED90
:108E9000D40497852C043B68F200861C21602CFDCD
:108EA000272CFE81C62F2C913A5008E4E3BA366F86
:108EB000F9EE3D628816B631AB76AE09C108C7221D
:108EC00000EE31A23688BC685BC31D2DFB52DF0962
:108ED0005C63D8A901FF443555AAAF04FBCC004C14
:108EE0006623711CC0356028A1B3D0FCC61A85D595
:108EF000516B90BD3CEE0C693B546390F20A6437B1
:108F0000BEBF3752DF0F1D43804709261DBB9D366C
:108F100011E2418B848191B21C7EA93FC10494B3BC
:108F2000EE809CBEBF5F237D5CE41895FA14BA679F
:108F3000618F57384A851914EA613727365D140264
:108F400035B3493A6EF3B19751EF9E6F7DECDA6A13
:108F50001FCC76654B66C9E42842354D21E7D67CA7
:108F600025F10400CC77718B43474D871DAAF896F5
:108F700054A610CC7BE0BC4E026F9F34B4EA3DF5A2
:108F8000B469A6EC07640D173A1137AB5E1BC491A8
:108F90002ABEFABB02F0ADB60727C89E9550B12095
:108FA000E3F857697118EFC945D97C45679DDE0C18
:108FB000DE6F2C4D05AD2563D040C72259D6BBE7E7
:108FC000A5BFC80A44B77FDFFFB821C38AD5D10740
:108FD000ED292AC3CC7CC7CEC955591FEA4C174886
:108FE00062D1B8DB7E84147A427FA3D1C5B0D1515F
:108FF000D897DD85A17585322DCDFF82C68B188966
:109000002801277BC70F4B0553A76E1F4DBA45AEEE
:10901000C9A345ACA3B7D8A38B6D206BD5363A88CE
:109020001903BCEA1225033AE24835479221017937
:1090300027C9910B944B9583FA2612D0D7E2503969
:109040007521C45D3F55BB857867434B56A4F70136
:1090500013EC456495FAF222D2D5B6219145C19020
:109060005550588FE4D9A86E3185F461A3B91EB468
:109070000116119D7653E97D8DC10A6A1CC8CA5D2F
:10908000BC1EF4C04DC875239267E6A8ECA86632F2
:109090002311289BCC117EAC5B9175AD054DB9CDEC
:1090A0001EE5CDA827A1D6C3D4FB3F7D581CBE1E0C
:1090B0009DC107F4E6F435267086B6EF366DA95BE0
:1090C0001F82F9240F3B2F50640DE0ECA49971B17D
:1090D0001B342ED0A64909A2FA529407BF039C0A5A
:1090E000859E638D13A66495E383C1BAC5F5FC0B19
:1090F000C6854895007BC1257FD370A2F3BBB01B0A
:109100003DBDD50DFF8B012A360815439C87186499
:109110008E63F2251587DF7298EC8ADCC14A77C02E
:109120006E2562CF124796F3717821F14712372BE3
:1091300068554BA4FF1E9720F7F63F0C759D67728C
:1091400068EBE5766E70F19511D295CE70779E60E2
:1091500043E4AC4D0F811D3170D80E0511914E6264
:109160007E244BF06B7C99D48D5EBCD9AE307B7481
:109170008ECBE10F48C2EBB866B38AA05950E0002D
:1091800066C845939B86F38E813AC61405C89ED760
:109190009823C513244D5C577EAB878506135C98D6
:1091A000D0E4884A8DAC8F1EADB84945B5158E53B5
:1091B000B9092F10813AEDFB402181BC543EC4FD1A
:1091C0002467BAE39AFF6B139F89ACDC238829B626
:1091D000B27180807FEC20007DF03E3E3A94061B09
:1091E000E2E750C07135F885B6035D7BDDA505B2B9
:1091F00065245A68AEB86C7B9C7D4A4AEA3DD5EB43
:10920000492BFE75E5CA722882EFEDADFE8F20DF97
:10921000BFC19DB6B86C68F634AC7B35192FF74DDD
:109220009E16194EC71E261DEF898E99E3442CF415
:1092300093F2D5B88DAAE015932EC37B0F4AB541A2
:10924000D99E5B50CB46ACC2D33B1E124BEB033DC9
:10925000148D6B05DC0F615672B4AF2CF74008AA71
:1092600011B4C0BC2F1D8848E00CFA68899CA5BBCE
:109270001655DAD5AF430081364A998BC43545ADD2
:10928000E794D1308BB480125AF652BD094C77E185
:10929000EF7CD65D93E5090E8CB30D1C2F14720C78
:1092A000FAAEC3F8E76A9258F5F6B91EB5A299D599
:1092B000600C2FA97ACB2FF824BECC94B2617BB17D
:1092C000D50947B5592D3104C8EDC07F98A859B1CB
:1092D00098E294EB3DF4DD22D4503DE4D26DBDD450
:1092E0000C5D9B7FF27B5606D56B4638FE7127DFFF
:1092F000BF699E9C82BB4DBF1DB02E808D2F5AE84A
:10930000D1FA0FA866B27F3E8645F1169980D21E2B
:10931000C24EF9AAA4C1C208A9E1E530DC8E8B04D3
:1093200058770D476D4B859584AFB90BF381B1FF2D
:10933000C38CD661A6C549840B72688C3D415EC45E
:1093400061430FE5C4FA311058C988CF166524CEA1
:1093500080E320A8F11CD506DA37CF9961F28D2C75
:1093600074CE4BCDF249118AFD20FB2F1314386CBB
:109370009974441E6EAA6B06A45F0E3A172F297DBE
:10938000E09C87EFB59BAE3914599C589F7C65A52E
:109390005B65B75AD60812E4C43FE45D39D63AEBB0
:1093A000E811E7B1661E433A0BB63D69C47A600F17
:1093B000D9C22989AA262928624683228FF1D51A83
:1093C0005D4CCAF3E5875273BB7BFC1013862A02FF
:1093D0003B20B9BB7E50CAFE6D128C6EA398070865
:1093E000DBE601AB4056FDEB28805A83D8700F02B4
:1093F000ED121EE2643F9B98AC1D8E2E4199A5B8DC
:10940000A620D9615E83EEE01BEE84EC8B445F9373
:1094100008F85458350D493A72FDBB88E8DE886972
:10942000763D2041D07FBEB8B070625034A1F53A8D
:109430009D493A50EAD9A588630D17B2F6C14ECCC2
:10944000DD00435AE8D5ADDCFC2D75CEAB2BEC33FB
:10945000C598B7A39175DE9487864517020EDF8401
:109460009EE7A0A7216A07FD0193107A17AFCF23CB
:109470004C739403F4B93147295078E4883492DA74
:109480002541582C850BA7D40A2B6102F1426B0DA4
:1094900054C2048E4256937E730E3E7AD8ACB010FE
:1094A000ACEF61CD289299985F012BE247DB1DA4B8
:1094B000B293E0BB24239107013E48ACA2CD903388
:1094C0002FFE6A4EB49A21834A31BE10349E8A26FA
:1094D0003DDE6B913A55DC6488ADE78ED14E157F49
:1094E000C4FE17DF030795A9B5BBB01CB85E61DDEC
:1094F000079E812AEEB7AAC4E1D9E343F619822B6D
:10950000F33844FB47D6B8CA4F87FEFE3B0D2CBD4F
:10951000BA1EA3A0DA472654B33B0D975258CAE6A9
:1095200030D1355E76644A06450CE86E9929EC73B5
:10953000BDC36824E81484F3F9348984A442812AE1
:1095400056FFAF5EEBABA43D65AFC82749A62779B0
:10955000679A79DDBE5A9C2CB5F7CFBCE506F6FCC0
:109560003179B35CE26309C6D9FF06446B42B5C4E6
:109570000B8D2D9E05144256AD0E615DDECDEDF5D1
:1095800029385B0ED87F092CAFDCAEA5514E33B81D
:1095900079DA590540BE163A1318C24946E09DAB28
:1095A00051E91A38A84B2A47EAE7B9D5EE586C8337
:1095B000CD4DBA2EF280188BAEA6310DA29DE48A55
:1095C000C741B8808758AEF9267F690FF19C0CED32
:1095D0009CCA61D4120DB44E7C955DE2CCCAE4C83D
:1095E000C6BB194E4EF41847E9D11D60A9FF410EC4
:1095F000D9CD397526ADBB12A37ED97E6692A05A0D
:10960000A7CFF0EBE67D92BC842278D0B191B690E2
:109610008E2B43E82A42AC7DDEBD18320EBD878812
:1096200009934BF4B038AC52C02253578E5FD5D556
:10963000743F63ECA37AD02D27725F6678E359B448
:10964000244EBFFC338E23AD596488BB0A2258DAFE
:10965000CBD147EC3E81F35095F66BBB8A9A1654FA
:10966000E30FF987919FD14A52F594904D7DE9C15E
:109670009C30B5D8845DE25D70346A3A3AEA4A813A
:10968000C817FA04749FD8BFB96CFFD17BB210938E
:1096900093849920175520E92B3D546A1000C8B9CE
:1096A00098B672364213BDB2D81EF6D4F80CA4A7F1
:1096B00035A009E726021250EEEB21427E947DD9B7
:1096C00046A82634C0EB1DDAA6CF5A35E9AA4AA32C
:1096D000D886EC53763EB875C1D4330E32A6220339
:1096E0007BFCB8786831CA18B7651FAD6E95F51563
:1096F000D3AC1EDE72AD3242B091EE092DE91A0DE7
:109700001D244A9FE97006F07E8FE0952D5DBF1EF7
:109710008F01002BB55F824F93D6A367C2EA8437CF
:109720007FF03F29E9BCC28889BDCEE940F101A89C
:109730009A9E2622A49BCE89239873B699E804E3C7
:1097400034949FC6346B679E26CD8EB979A4096682
:109750004B1339AD5475487AA5C1B17C6371263E6F
:10976000274B91140CC7A6F90A80EC2F438777EC9E
:10977000683EBCAD948E96DC556E1D37F9AA3FF558
:10978000A3E6153B29C620BAB35718D8D06824E100
:109790008B339BE84E5AF93EBC7B40B863638B4DDC
:1097A0008709A83E1540AB6C84EE74AC3A4464085B
:1097B000150A7FF9643EE8BAC1A21C6E6CBC7C63DA
:1097C000B87DD0E3DBE325A90501F53BD6FD89B9DA
:1097D000727AF16827A9729AB929484981F0A9B724
:1097E000B6521ECBD65783EAFA1E93EC6EDB6A8F15
:1097F0008FA9DD3F20C42DE15A87311776A27D263F
:109800007F594810125EC46A0B348B486A25D7A171
:10981000C2DC8A17D2E1B071C23642BF26046B7B2C
:10982000AD0E3E9EFFD419E9000DB4AB1EB82A0759
:10983000EDA3FA9BB638B814E802A017DE11252B69
:1098400075949D197784662F0656C095DF65CC14F4
:10985000A0B428FCED3C3364C1EDB9677FDFDE8E38
:10986000DBD5450B8C9441C9A517059EBC98BE8DD0
:1098700094FAF099A0415AF6D53162F697BB0016DA
:109880007964F23794F9A782874D87AE684ECC662B
:109890002997A910C72D6A18E73A2A2DCCC8F726B0
:1098A000BFA639471841044EB8BA1A51C4E9DCF5CD
:1098B0003D2DC301F7D12555764FDA3741AD23173A
:1098C00010AA853CF4F043F3FE045E67D7CF6C6FBB
:1098D0006AECFCF0812D9A079F0C4458D6734F45D3
:1098E000A11A585F370695EA2EA6ECE1B625DB5F94
:1098F000E0BC551551620455DBB05D5ABA968B75C4
:10990000FD90C22CE3635537D5520B76541258980C
:109910000A6F006E02137428682A05666EC28A20D8
:1099200058A3C6A907EF561709AF5E02200A47DA07
:10993000E800B02BF267FF7610144DB31B882D3B67
:109940001C7F3998B0388676C510A0F424EE86972F
:10995000598531C4DF7D97F73C963EC290BBD67ADD
:10996000B6E6A8E89477F83A2B0E4DD17386741EAC
:10997000B1A798F3056EECF5DD45B973AEB0C1241F
:10998000EFE3CC0AB41E8B8CC4E88E52771FC3253C
:109990006712579B40CBD8451C744635A33773C21A
:1099A0006880F94E7B7BB21B6A51C8CBA29EE399BB
:1099B00044BFBF1362C341F21629092C2CF7454D51
:1099C0004A87DE5B43041E7447759D98D7133C5647
:1099D0002AF3A2A92DE1F2A146DF2968897B9163D0
:1099E0000F456DC95249F42E09E6AE4D98C1ED7F81
:1099F0004D87553691EBEDD05D88601FEBE3291F55
:109A000014B810644905AE40910F9C17436A0BF7D8
:109A1000046C25A63F92A1DB59EEC69AE02E80A3E6
:109A20007D5D9B574B843FE81F193ECB69E9DD55AF
:109A3000EEFFF431BA9BF89E6599A19DED21D50307
:109A40005C6F67B22FEC2818E8AFBE97476E8F7631
:109A50002C7B2E085416A0AA1210D0675CF5F40CCB
:109A6000A9F1CC091DBB6AA07F15EEF02F1EF45A98
:109A7000A3767A990A48331A9D15A6C247D8F2CA26
:109A8000DF69EC8215562F747BC8EB650F64CB6AD7
:109A9000CB864B51702DD173AB121E8411BCA983A0
:109AA00021226C77524C6CF6BD7DA3769CD17A1C3A
:109AB0004E94636E8DC9EC22EC6C3EB9A5886CA205
:109AC000D64F159C1D5EDD6781EB0B8ADE3A9A50FE
:109AD0005B8F3CC0B4468B79EF91489F3546979198
:109AE000F57412E8E1F990E7A21F1BF71092437E8C
:109AF0007B809419F7E352F828B6EC2A8DA833AA94
:109B0000E0991B7F73D8A15BDCC11AAD994F0B465E
:109B1000B3C1A9581DD7AEA73D31C1D70A08BFFAB6
:109B20006B82D569E60DBD11DE3194099F54254E37
:109B30009BA8A887B78BC56465D228C2CA0C225ED1
:109B4000C0FA46DA6886DCF4A202E6AEC466C09DBE
:109B5000F08D6C59EE600D1B56E231D063B14B1A9B
:109B60009331F655C9D9E3A87039DD6CC702D659CF
:109B700028888BE1F17601C94B71A51A34D269BCF2
:109B80002460F2AE0F147B71A0A44BAA85F6A9B590
:109B9000E874BE6A9F1BA8F864015811E228B599C1
:109BA000ECA24382B0F7A1BB8A90E4CDAA2488ED51
:109BB000DD8D0D7C38801994AA338BEE72F422DE91
:109BC0003E34616145508D7F162C8A7618E5E6019A
:109BD000BCD76E1C9CE16F30FB56884E9BA76EFB7A
:109BE000323868FEF08D9BA719B0002959D55AEA82
:109BF0002080DBA65DFB5ABF68C2DA1DA144363760
:109C0000E83F0619016FD220429F55BA091B26CCA6
:109C1000BB0DFA180E5A032621B0CCCEB452A4E8DC
:109C20008BF806FCACA1F3AC9AF63AA82BD61EFF33
:109C30002B4F8504CCCC44E7D33374195D57F6948D
:109C4000EC4B32892251E2EFAA14F33025FF911533
:109C500053A82CDC61AF0A9AA53523AB9B10397D44
:109C6000961F7900760CD69361325B384B2DCE135C
:109C70001342D816D2263F54119DFB5B8156480FE4
:109C800090F81A4D24A4B605297785E282C0CA1738
:109C900061AC9958D4AC5EC880DD13EC99768DF137
:109CA0009DF9BA024BFF6552426CFF69AA569C743B
:109CB000A964E6099029FADC03CBFF649ED0A58352
:109CC000D74F18B8765123C6A649DC588E78E3B82A
:109CD000BB672DB6BBCA19D45404251C78A0E77AFB
:109CE000B52ED753C76C236ABA40E5AE06B19CAF18
:109CF0003208525E5BAB4DA317049AEEB468CE5B9C
:109D0000ACBA1B458AAD56B7237AF4C8BF7FA559B4
:109D1000A918E5CBB9ECA6B71E5EF7F5B7F2C8D423
:109D200050D2906D0200B551EC088F0BB358898A60
:109D30000725BA5057DF0BF0B259B3A0FFE438D86B
:109D400009798EC626A21FB6C57E7F56A55A1DA1CB
:109D50008583DB134133785D4EEA0E4088D9E347B3
:109D6000977751FD1800B29B799D40993FF9AC055A
:109D7000EE941F71F35B09DDE6F534EB755FF17668
:109D8000DB1292919BBCBD8E78753E35BCE290791A
:109D900085425EF7F42494FEAD14A957B664A0681A
:109DA0009220F7B4B2F430C0CEC90E164B1354A9AA
:109DB000C5D4BC2FCF54CB12CE1B5507DB02D8D253
:109DC000291914D09D0991A8ED25E6BE7BE8C5B4FC
:109DD000B630F867A128065FBC9F9296EFD2B4BB5D
:109DE0004DF475119377B62C22394BEF0B368CA4BA
:109DF00051F98A5AEEDBA3472442A2340905809226
:109E0000B95B3D9E5F6A6E420AE16E29FB8BFE0CD8
:109E10009843EA1F732B334DF768EAC67A421F074F
:109E20002EF3A169A2914AA71340CBA279D7146C53
:109E30001FF2D35E4FFA8E56C65A8780B050891CE7
:109E400037F3AE1E1F9F98A8834D70F1C97F1D0F79
:109E500082AA26A203DA0C53F4485DFABFCFB86891
:109E6000AD90E544828F9ADBB2497CD4C6FBB684C0
:109E7000AC577E650ED4AC1C184284F1E0C538B5F1
:109E800094AA0C10204CA0773C0A7D27024763ACB3
:109E9000A32D4F73488CE523DFB3E9F5DD386A1550
:109EA00035DE0ED964A5B6B2EFD72580216E66C522
:109EB000A3181CF79A0E7BCF8264E500C662B9F046
:109EC000441BD899D5776B21417B24BAE14DE252EE
:109ED000F41A66318BFC65B294D0537AA66E28D9F9
:109EE000A45BDC88A527956BC0960643C5B8DF6FD9
:109EF0000747C8C13C3DCB2FF65D3F79B537863467
:109F00004758CA064243FEC1E61BA1401637E44A41
:109F10008DA300915262FDF8348CB9D1D08E0C78AB
:109F20003554356A4931F794F9D0DFBE40AEFF159C
:109F30002D0802D4569E2BF6F58BAA213963BAC997
:109F40001853848D71ED22A9386383280745374B58
:109F50004A9BB30639BEC67C4CE68ED27E5661C49F
:109F6000368BA34860846136BC4E93191FC063AE24
:109F70008FB08267DD2DB5CB2094A24301475E6C84
:109F8000E31BE6736DA6F6D48A3F63EE87F254397D
:109F9000CD8325E78654CB856C12B86BF1356E1DE9
:109FA0006F5AB1A3E7C445E543EC67AA19613B8545
:109FB0005B65D0762F5B4ABEE4DE940A2AD784CD57
:109FC000E7EA1893F664622958B50724ACFA6526C7
:109FD000B275310D1E246B381D6E794D54F202336B
:109FE00087718690C85EF1FE29BC69706781698BB4
:109FF0001E816381082196B5A5E8DB2480FFE1DAA4
:10A00000AECF36AEBD1D65138083D211175190F7C8
:10A010007E915E1F72209F506697FB1AEC24B69EBD
:10A02000AF888445A80D2532B970310A3F4E5915C5
:10A030008384BD43D1640EA5BD0B306731135FFB34
:10A04000A3A8B6CE96E6F59DB5CE670BF73D2D6776
:10A0500067728F3BF319DAC41AE02FB5ED8152FB1A
:10A06000E25F9B730E9DC7745650E4AC084574BC08
:10A07000F96B822BC751D77E548034AFD5EBB01823
:10A08000F33D2DBAB97C095F7C3A37E3D2E7DDFCBA
:10A090004524C6FE96FA99672F3DD6B5D27337632D
:10A0A000CEABEA9A3012AAC287EDEAEB448FC44ADB
:10A0B000662AC884C7734F04D8C72D664A7DDE65FB
:10A0C000083C3AA7BD455A73E1A3C7DF3E536C6114
:10A0D000097B4292450E764868FD58398102052871
:10A0E000B9EB71CCC3E40220D9268E4A77E013ED98
:10A0F00001DBC6CFC01013AB186C9C0F4DCF9E7008
:10A10000FB8DBA2C7100FF079626AE4CFC1C631A1F
:10A110002E8A88B1264E333ED1B2B8B8EE5C0B928F
:10A1200072872D4B7AB3F2F0EAEA9DD81BE171E811
:10A13000CD1D36939E6910AD55CDC314893D9D6AE2
:10A14000C89658412ADC6DAA57790B411CFF7D182F
:10A15000C7645453B4C8898D8457E6AFBE441735DD
:10A16000BFE2665A2CC8CAABB1E3D1C32135BA30BD
:10A170000FE64D383237BD18DF601B1C72B1C9A421
:10A18000E9DA8860C27513A2301F9E7B9EF2271AFF
:10A190002EC394D5E27B6665E01287340C9B8791D1
:10A1A0005F97830603664F75AC953038F6D77D44CC
:10A1B0005D916C63458F32D1EF474583FB53BC31D2
:10A1C0008E5C7BD25FB7896F1F466172F651D3A850
:10A1D0008935647B05ABD0DC2745745EC7C188E850
:10A1E0009276F841BE4EC9E41A6BFF243BA6326159
:10A1F000A86F0A2ACF17A44F13D53EAEB5F34E630E
:10A20000AC2DE1679E26696C4A8A70812447A94972
:10A21000DF7ACA6BC572C60CCFC2CBB357B74D0934
:10A2200067E8D4906D8C2AC1AD70B876D240666470
:10A230000FEC337BDF20330753B4A743555378A784
:10A2400027BCC0B7DB14AD4E0F04837A7502ED59FD
:10A250000BA1890C4FBFC7A0FD310CA4A1B6EBD553
:10A26000314AB2CE010F4E9D0D5241E08DF33910AF
:10A27000D01386246606BFFEF8E694C41D14BE40C3
:10A28000E664E1659E238BA0FDF138B00248739D22
:10A290004EE9E0AED4366AC485C3C4FBA4DB676074
:10A2A000371D6DA4D5FFE8030C8321B66270DA8CEC
:10A2B000887203DBBB0ACC806BE1458EA66BC2F6CD
:10A2C00068DE2DBD2A3E20CFB04A127F31569CA4B5
:10A2D0006B6BCBC2306B38056AD8CA48CB5A8D1528
:10A2E000B741B336B03B86B5E38CA9D5A5E8AE2718
:10A2F000DB7F3A41CDD646CA693DDFE6AA0EC18A68
:10A30000F4CC6D02E95DEE7E89FBC7DB1593B2806C
:10A31000DA07E93EE2CE1073715814EABAF484E029
:10A3200027DD57AC07864D8B3EC720BC71D731C3A4
:10A330002275AF1E62768D7CDF93BAA30DB4C11374
:10A34000EE3B7D13889F750D981B2180090DAE345F
:10A350002E7B8447CE88FFF7B271548F04BA4C210C
:10A36000CF0EFCE04CFDFB1F96D2C96BA0D7FE615F
:10A370000BA3EFEF200583C34D259FE278C0BE52AB
:10A38000E04DC3000DFCB528E40D98CEE955191831
:10A39000D64D7FCE1CE0B6064D835B98623C3519E6
:10A3A0007449EB5E1A26E4EA5027E966E926217231
:10A3B0000C4E3451BC73FE794B28F26FEAD4AA9A42
:10A3C0009E944144AEA1E0B2D36DD1C2281EFE9B43
:10A3D0008B294C7C499AB8B62E1D1A8E3FBB2E860F
:10A3E00093AD21D3C129715D414BE590D5E1FBC10E
:10A3F0001067E955085D55D57621D8BF8BA0C97F78
:10A40000AB977B2ECC737341B840A4D769FFA7EC00
:10A41000081F2D8C44BDF18CE9BA6FD9A4E68BD10D
:10A420009C72512B38BA1CF201B1C6CE698B0E84D6
:10A4300073B521F9BFFFA7E96A64EEB13F75CF3F5D
:10A44000EC8740B0A3563E2E4D336F6F9B7E77D086
:10A45000B79F0BD9CFA48EE898814723B5F3CE746C
:10A4600020D657EB7C375528A23D416236BCE43BF1
:10A470007220EA4073C0712922DC5F565242D375C4
:10A48000F73A8464C5E7445C851F72A372393812B9
:10A490001AC35DB4F06699666474A58CBF6DEAD684
:10A4A00065D1C02F9DF7E2DA4D382743394940C0C6
:10A4B00056B3F9912B8BAB252AA0F1A8C14CA07DF6
:10A4C000937940DC288CECFD5F6A437B396BE2F7C3
:10A4D00055413A8E56EFC4F8E6691B7B51B7021915
:10A4E00000C9B73EFBF1CF48CF6AA7AFBA12A22787
:10A4F000CB633246C26C6D70BC4C90D929DFAAF098
:10A500007198D326B008066CFDA87876E47A515F7E
:10A51000BD19AFD083237E6B6D26CD3AA5C384A52C
:10A520007203D04760E675498E3E9A4DFBB79D7227
:10A53000703E29E363330BEEDDCB477F3BDB100935
:10A54000EDEF96B9689B577DF594EF8937B082DDC2
:10A55000F301D89F6549B687D2A17ECA10E6893932
:10A56000F3164C3F28145F1A8AD4C9CF485A26F8EC
:10A57000427BE53A7EC59C81F39A09291074DDA2DD
:10A580009503EB6DB61CCBAFEAFA95B1A7094AABC0
:10A59000FA1F4CDFFF220EA346324FF3F89C30EB3C
:10A5A000CE21669C9229D7B4F492534C07E04463C1
:10A5B0004F9220D280463F5BFB58EBA229C2245029
:10A5C000DFC8178591003F4B321E76952E3BD2F5A2
:10A5D00018F80F870AC1B0F2285413A209F86DA029
:10A5E0000F478C643EC12C95D75EF19218CED6A150
:10A5F000E16999D6BDF7BF52B23CDA364B38FAD290
:10A60000BF9333D12599743D3C27A2E558BD877986
:10A61000EC4B76F9273623561BAAC4349001618788
:10A62000D70CDBD65578A2DA9F1A352E920710A2E6
:10A63000EF9FFF83C1DAB8AD9433D6A2F707ABE63C
:10A64000D907113DAE0A33E067C94814E85FC0F688
:10A65000FC5B91D4F8314C2A5C3863CA212C034945
:10A66000E7CA8BDF90521E04382696AD732AB218C3
:10A670009B852ECBB47D9C88D325229F1F310179E9
:10A6800086AAF83E00A3301C6FF81E71F39AB44AF4
:10A690001177F1187C8336A3AA0128BA84D2687195
:10A6A000BE5E85E1EA853B7A4765D6509BA8709FE0
:10A6B0007C7B53284F5A60B37516FEF1B4E50A054A
:10A6C000ACB681A2A1498A125BECD7FF8EE49684D6
:10A6D000C10BF3D15C9E19382CD3208D5CD2124C67
:10A6E0007D42A076E19741E0916BDEBCF769CCFE3C
:10A6F000EE13674724707181F714EC25650150BB98
:10A700005857A34D481F0C6EA1DF030A633144E282
:10A71000C0D36F9B301E0BFFE5DE3724ACE3A0E215
:10A7200000EE91E4D69216297C489167BE6B40B248
:10A7300043E20976CBBEF8EC186F0A5A35A813F637
:10A74000C36C0A83E1499A8A7BA8DF65836B59C988
:10A750004D37C89A0DB4E32C061E9DEB62CB126EEA
:10A76000AFF852AD7FDF9C389BD05E31D57A16862C
:10A77000F3FFE5C4270C001B48A409427087D29B55
:10A78000F4B71DAFC072B33A06C9DF76EAFF1BEF1C
:10A7900031BD5CE5F49B9FAE21F0DE6DD7058E2BBD
:10A7A000036FCF1475FFB02D0AAFAFE51947BADEBE
:10A7B000DE39966FBEF91422375F2F8B2D5367A8B1
:10A7C000D15682F838AD3DE6F5A2FCCD748AEF3F54
:10A7D00015E7559704346D702264E2AD4C5D3CB4CE
:10A7E000409E8165E20A77BDC98D67986F8D6A1BAF
:10A7F00007BA3ABED9CAEA42AA892A9D0FAC349A4E
:10A800002C63053D877E20EC51736E5610A55C329B
:10A81000E6D57DC760168DEA6BA1E307A658A37342
:10A8200068ED7FC13ADF22DE58DBA2730DE3FB68DF
:10A8300000154028DC6F7BC39626CF76DB026BF1D8
:10A84000804AEC6E0D5A36AB1050A9C84B687BDBC2
:10A85000404B795F718D241A462C5A657CD731485C
:10A86000F8F8FC883FC2F24BD4F5CD861CFC189B4F
:10A870006B1822643177D49C3D74C4BC3D4B04B347
:10A8800045B94F8050F4C09DDF870B1147E9B5C62D
:10A89000BB6F05427EEA8A37365A7031F698B80D9A
:10A8A0006A28575540BB023245ABDD7A0FF96EF18D
:10A8B00086D474892424F6D765D1D5638D93758C9D
:10A8C0004F70D63C3A279754BB8CAF9A506B0B6DA8
:10A8D000C7BD95A286376EE5F5FA81ACDC86F660D9
:10A8E00009A9B16234A52E05ADAD736FBEBF83FA61
:10A8F000F3A331E3535029C4D271288CBCDF1E0866
:10A900007D66C79A4D8FC450B593230DFD670EE742
:10A9100033C432151EB26E5023913256C6D4B4FBE6
:10A920006C24749CFCF3664CB31A125DE9D46EF887
:10A93000D537EFB0B72F53403FDAE7EBC29B5C3916
:10A94000683328A94345E6DF222EB617C08910D800
:10A950008AAFDA7A6DE6FB7667AB0ABDAD22A9361F
:10A960005C1F165D7EDE2D4E6ACBE1BD467AB8D304
:10A970004402BFF4C4FC4399AB650E5419B2127A79
:10A98000936FB6B96E191858EC0EDE181A5565BFDC
:10A990003946498CFC469771EF2A77EEF20D311A51
:10A9A0004ED5EA9589D84E508F883F9D462A869E7F
:10A9B000A56AE1ACCFFF91672D3E689B4604EE3F50
:10A9C000BDEA1B784311CF1E6F990CC757DAF73ECB
:10A9D000351BDD434FE806B603FBC4AFA90B427439
:10A9E000570F527239DA4C17F98D2E6687021CB553
:10A9F0000473BA4CC3CD1EED2501732CB69BA40A7B
:10AA0000BCD23AE98764FB776BA807617E9A15F49C
:10AA1000E84C1369FDFE503401186048464B749EA3
:10AA20000AFEBED869573CB2300DDCD3B30E48EFF6
:10AA3000D15FCB2F4E714F299BCBD22247EA7606AE
:10AA400043B550AC963C6F45D4781C1885D324C6CA
:10AA5000AC4F1CCDE05DAC7F16DFCBEEBFAEAC944F
:10AA6000B39FF7E43DAB0FB60A8A570BAE95010FC3
:10AA700076B89FCB331C9D8A9B067A08F04E537D97
:10AA800035E8003D1F79CA3C338600F16A9497444B
:10AA9000BC9C167A7B05292F90B0E7D36322330F35
:10AAA00051FFFC60107BCC9F3606FCD778C4B21AED
:10AAB000F5EB12606E65CE94FB9D1AB8335BE4F43F
:10AAC0004906CBF0CE1D57A2A05A3941EA9537D698
:10AAD000984C9996E9080BAD3FFB34F2AACE9067EB
:10AAE0006649A3F3605C78328F31FC142141AE7F5C
:10AAF000CBB662C8BD8214241B4FAAB1187384CA96
:10AB0000ED3C43A06FEFFF3B2666F8FABB26599653
:10AB100086147DCD69D0A42BB5D71E6F867F66893C
:10AB20000B30F5FE96447E4B411A4455D7ADF0806C
:10AB30009FAEDA443EEA2E191466EE4F8F54AC6D88
:10AB400028EBADEFFA0BB5AB8FF4B5A134BE997419
:10AB5000AC293A7BDCC8452D5CEF430A834B80046B
:10AB60003E4DBB2D439F0EF7535752E098F81B798B
:10AB7000E1A4828767C11BAD1457CC6E40F440E35B
:10AB800031E0278B496B609CD8E110C67D5BDEEC21
:10AB90004FDFF02D4832F6DD6AA336EACA7ADC656B
:10ABA0000A6E0525B9B68CA5B50B4C377381C0CE9E
:10ABB00062BC19BAB338C52D3468D8402274E7088E
:10ABC000B508F0D820DA6ACD23FC88D128724B84EE
:10ABD00009DD850D24E5AA5461918A35749EE5E36B
:10ABE00004990C5C7E7119052A720978F5DE368E9F
:10ABF000B75B569CF1D5F793A27E9777414CCBD0AB
:10AC0000E8C5C4F98116682BF1BF5C504E7D8B44BA
:10AC10007CFBF1278C5320C8E41AA7B23B7A5D0471
:10AC20007EDF233028460BCF9383696B3AFC82CEBC
:10AC3000F1AA9CCA87041E460304050A08060BFFF6
:10AC40000209070D010C00FF202020205F5F7C001F
:10AC50004D454D4F525920434C454152002C004424
:10AC6000697370206F66660D0A0055534552006780
:10AC700000424547494E0052414400442E4D590080
:10AC800055534552202020006620200067202000D8
:10AC9000424547494E202020202000524144202098
:10ACA0002000442E4D592020200043202020001C4D
:10ACB00017171717181D191B0100000101010100CA
:10ACC00000081C242C4448586C74000306090C0F1F
:10ACD0001215181B1E2124272A2D303336393C3FEC
:10ACE0004245484B4E5154575A5D606366696C6FDC
:10ACF0007275787B7E8184878A8D909396999C9FCC
:10AD0000A2A5A8ABAEB1B3B5B7B9C63000C6310085
:10AD1000C63200C63300C63400C63500C63600C68B
:10AD20003700C63800C63900C64100C64200C643D7
:10AD300000C64400C64500C64600CC3000CC3100F9
:10AD4000CC3200CC3300CC3400CC3500C03000C055
:10AD50003100C03200C03300C03400C03500C036FE
:10AD600000C03700C03800C03900CD3000CD310000
:10AD7000CD3200CD3300CD3400CD3500C13000C11F
:10AD80003100C13200C13300C13400C13500C136C9
:10AD900000C13700C13800C13900CE3000CE3100CB
:10ADA000CE3200CE3300CE3400CE3500C13600C1E5
:10ADB0003700C13800C13900C12E00C300C300C331
:10ADC00000C300C300000306090C0F1215181B1E58
:10ADD0002124272A2D303336393C3F4245484B4EFB
:10ADE0005154575A5D606366696C6F7275787B7EEB
:10ADF0008184878A8D909396999C9FA2A5A8ABAEDB
:10AE0000B1B4B7BABDC73000C73100C73200C733CD
:10AE100000C73400C73500C73600C73700C7380041
:10AE2000C73900C74100C74200C74300C74400C735
:10AE30004500C74600C83000C83100C83200C833DA
:10AE400000C83400C83500C83600C83700C838000C
:10AE5000C83900C84100C84200C84300C84400C8FF
:10AE60004500C84600C93000C93100C93200C933A5
:10AE700000C93400C93500C93600C93700C93800D7
:10AE8000C93900C94100C94200C94300C94400C9C9
:10AE90004500C94600C43000C43100C43200C43388
:10AEA00000C43400C43500C43600C43700C43800C0
:10AEB000C43900C44100C44200C44300C44400C4B7
:10AEC0004500C44600000306090C0F1215181B1E8E
:10AED0002124272A2D303336393C3F4245484B4EFA
:10AEE0005154575A5D6062666A6F73767C7E8084C7
:10AEF000888C9094999EA0A5AAAFB4B7BABDC3C8D8
:10AF0000D2D6D9DDE1CA3000CA3100CA3200CA3314
:10AF100000CA3400CA3500CA3600CA3700CA380031
:10AF2000CA3900CA4100CA4200CA4300CA4400CA22
:10AF30004500CA4600C53000C53100C53200C533E2
:10AF400000C53400C53500C53600C53700C538001A
:10AF5000C53900C54100C54200C54300C54400C510
:10AF60004500C54600C30044535A0049535A005394
:10AF700051525400312F7800528B004C53542058BA
:10AF8000003E003C007888300050534500783D7901
:10AF900000783D3000783E300044424C2A00444264
:10AFA0004C2F00C300C248455800C244454300C26C
:10AFB0004F435400C242494E00C9CB00C94900C7A3
:10AFC00049005753495A4500783C3ECB00434C4515
:10AFD00041522052454700454558004F52004E4FC0
:10AFE0005400414E4400584F52000004080C101405
:10AFF000171D2024262B2F313335373B3F43474B3A
:10B000004E5154585D6064686C71767B7F83898C87
:10B010008F92989EA2A5A8ABAEB2B6B8BABCBEC07D
:10B02000C2C4C6C8CACCCED0D2D4434C58004845BE
:10B030005800444543004F43540042494E00528C4F
:10B0400000454E54455200C84900522F53002E006F
:10B05000783C3E7900434853002B002D002A002FF6
:10B06000007888790078867900783C3000783E79DD
:10B070000052544E00CACB00CA490023420041424C
:10B08000530044424C52004C4A0041535200524C2F
:10B09000430052524300524C436E005252436E00E2
:10B0A000783C3E49003127730032277300554E53D8
:10B0B000474E00534200434200423F004D41534B34
:10B0C0004C004D41534B5200524D4400534C0053E1
:10B0D0005200524C00525200524C6E0052526E00BE
:10B0E00030003100320033003400350036003700C4
:10B0F000380039004100420043004400450046004A
:10B10000CAAC0000C5AD0000C5AE0000EAAF00004B
:10B110000AAD000005AE000005AF00002AB0000037
:10B1200000000000FF00000010B1000000B10000AE
:10B130004040404000080F151A20262B30353A3F7A
:10B1400043474B57494E444F572000464C4F4154BC
:10B15000200053484F5720006E2E642E0052434C5F
:10B16000202E0053544F202E004C424C20004754B8
:10B170004F2000475342200052434C200053544F6D
:10B180002000286929005346200043462000463FFE
:10B1900020000000FCBDFF7F010000005077000090
:10B1A00055770000647700005A7700005F77000051
:10B1B0000305000001000000FFFFFFFF4D0000003D
:10B1C0000F000000F4010000FFFFFFFF6AAC000069
:10B1D0008F7900006FAC000071AC0000A17200001C
:10B1E00077AC00007BAC00008E7300005B75000044
:10B1F00080AC000088AC00008CAC000090AC00007B
:10B20000A17200009BAC0000A2AC0000AAAC000040
:10B210005B7500006AAC00008F7900006FAC000025
:10B2200071AC0000A172000077AC00007BAC0000A4
:10B230008E7300005B75000020202020202020203D
:10B2400020200000030000000401030102010104AA
:10B2500011040F041704160118010502050804085B
:10B260000B0804040501050409080904060807027F
:10B2700006020402060106040701030803040C0881
:10B280000D020C0203020C010C040D010D080D044B
:10B290000802080807080202070408010804090256
:10B2A00009010A080B020A0201080A010A040B013B
:10B2B0000208020410081102100211081001100403
:10B2C0001101120212011302130812080F081204CE
:10B2D00013011304140214011502150814081708A9
:10B2E0001404150115041702170119081A0219028E
:10B2F0001602190119041A01160816041B021B086C
:10B300001A0818021A041B011B04180818040B045D
:10B310000A1409001D27FF131EFFFFFFFFFFFFFF99
:10B32000FFFFFFFFFFFFFFFFFFFFFFFFFFFFFFFF2D
:10B330000B1508011C26FF121FFFFFFFFFFFFFFF79
:10B34000FFFFFFFFFFFFFFFFFFFFFFFFFFFFFFFF0D
:10B35000FFFFFFFFFFFFFFFFFFFFFFFFFFFFFFFFFD
:10B36000FFFFFFFFFFFFFFFFFFFFFFFFFFFFFFFFED
:10B370000C1607021B25FF1120FFFFFFFFFFFFFF39
:10B380000E18050419FFFF0F22FFFFFFFFFFFFFF4D
:10B39000FFFFFFFFFFFFFFFFFFFFFFFFFFFFFFFFBD
:10B3A000FFFFFFFFFFFFFFFFFFFFFFFFFFFFFFFFAD
:10B3B000FFFFFFFFFFFFFFFFFFFFFFFFFFFFFFFF9D
:09B3C0000D1706031A24FF1021E9
:00000001FF
